:10678500011300000501013C0200000301FA0400A9
:10679500FA0500030A0A5A0B001E0C00FA0D000345
:1067A5000E00030F0164100096120132130AFA1449
:1067B500010215000217010A1801FA1905321A011A
:1067C5000A1B01FA1C05321FFFFF20FFFF23011ED4
:1067D5002400642A00FA2B00FA2C50782D003D2E57
:1067E50000462F001E3000643250783432FA3501ED
:1067F50064360164370150380A643C00643E003C4D
:106805003F000140FFFF411450420A5A430AC84461
:1068150005324500B44600FA4701784802034C00AA
:10682500FA4EFFFF500505510596520A32530B46A5
:10683500540A96560102570546580002590A465A07
:1068450032FA5B010A5C0A325E000A5F00FE61FFF4
:10685500FF64021C6600016701016A0A3C6B0000C7
:106865006C32967300007400007801327901327E33
:10687500FFFF81FFFF84FFFF8500AF8600018700D2
:10688500FA8901088A00009900009D0A969E000178
:106895009FFFFFFAFAFA00000501013C0200000320
:1068A50001FA0400FA0500030A0A5A0B001E0C003F
:1068B500FA0D00030E00030F016410009612013259
:1068C500130AFA14010215000017010A1801FA1932
:1068D50005321A010A1B01FA1C05321FFFFF20FFB2
:1068E500FF23011E2400642A00FA2B00FA2C50789D
:1068F5002D003D2E00462F001E30006432507834A6
:1069050032FA350164360164370150380A643C00B7
:10691500643E003C3F000140FFFF411450420A5ACB
:10692500430AC84405324500B44600FA47013C48CD
:1069350002024C00FA4EFFFF500606510596520A18
:1069450032530B46540A9656010157054658000125
:10695500590A465A32FA5B010A5C0A325E000A5F3E
:1069650000FE61FFFF64031C6600016701016A0AFE
:106975003C6B00006C3296730000740000780132A5
:106985007901327EFFFF81FFFF84FFFF85FFFF86D0
:10699500FFFF87FFFF8901028A00009900009D0A19
:1069A500969E00019FFFFFFAFAFA0065006F0079D5
:1069B5000083008D009700A100AC00B600C000CA9E
:1069C50000D400DE00E800F2005B0063006A00729C
:1069D500007A008200890091009900A100A800B00A
:1069E50000B800BF00C700CF00D600DF00E600EE0C
:1069F50000F600400046004C00520059005F00655B
:106A0500006B00710077007D00830089008F009581
:106A1500009C00A200A800AE00B400BA00C000C6E9
:0E6A250000CC00D200D900DF00E500EB00F14C
:1035E70090006AE0D3940440149007DAE0FEA3E069
:1035F700FF906787126B6CE493F59980129007DA56
:10360700E0FEA3E0FF90689B126B6CE493F5999042
:1036170007DAE0FEA3E0FF906785E493FC7401936B
:10362700FDEFB50507EEB50403754E009007DA12F6
:103637006B532275A71085F97385FA747E017F0095
:10364700E574126B45E5732FFF50010E8E5A8F5BA1
:1036570090001FE0FCA3E0FDEF2DFDEE3CFC8C5C31
:103667008D5D22E55DF5FBE55CF5FCD29322E55D1A
:10367700F5E9E55CF5EAD29422E55DF5EBE55CF565
:10368700ECD29122E55DF5EDE55CF5EED29222E50F
:103697005DF5FDE55CF5FED28722AE5AAF5B740699
:1036A7008E048F05FF126B358C5C8D5DAE5AAF5B58
:1036B70074068E048F05FF126B608C5A8D5BE55B79
:1036C700455A60137406C3955BFFE4955AFE8E5AFC
:1036D7008F5B785C126B99E573A85CB80015D3957E
:1036E7005D4010E573C3955DFFE4955CFE8E5C8FCE
:1036F7005D8010E573243CC3955DFFE4955CFE8E09
:103707005C8F5DAE5CAF5D743B6F4E6006743C6F63
:103717004E701AAE5CAF5D743B6F4E7005757301EA
:103727008003757302755D3A755C008003757300DD
:10373700229000AAE0B40104C20E8002D20E9000CB
:10374700ABE0B40104C20F8002D20F9000E8E0752D
:10375700F0DCA4FFAEF0740A8E048F05FF126B3500
:103767009007D0ECF0A3EDF0A20B401674038C0683
:103777008D07126B4574011200399007CEEEF0A346
:10378700EFF07E017F009000A6E0126B459000E904
:10379700E08E048F05FF126B35740AFF126B358DAF
:1037A700609000F2E075F0DCA4FFAEF0740A8E04BE
:1037B7008F05FF126B359007D4ECF0A3EDF0900066
:1037C700F4E060139000F4E0F5F0741684FF7E00D7
:1037D700EF9007DEF0800674649007DEF09000EA51
:1037E700E090008FF0900134E0900079F09000C3F2
:1037F700E090007BF09000ECE090007CF090009867
:10380700E090007DF09000DEE090007EF090011ED9
:10381700E0900082F074E390008EF09000D3E0B463
:103827000B0874E390008EF0805A9000D3E0B4192F
:10383700129000E9E090699A12008CE49390008E50
:10384700F080419000D3E0B41E129000E9E0906947
:10385700B812008CE49390008EF080289000D3E09B
:10386700B428129000E9E09069E212008CE493908A
:10387700008EF0800F9000D3E0B446089000CAE0B5
:1038870090008EF0900092E0FE9000D0E0B5062701
:10389700900094E0FE9000EEE0B5061B900093E0E8
:1038A700FE9000FCE0B5060F900095E0FE9000A3A7
:1038B700E06E70030239DB90006AE0C3940550089C
:1038C700740290011FF08006740890011FF09000A9
:1038D700A3E0B401067400900109F09000A3E0B4DE
:1038E700020674009000EEF09000A3E0B4030674A3
:1038F700009000FBF09000EEE0D394014014741A9E
:10390700900121F074009006E4F074009006E5F051
:10391700800C7400900121F0741A9006E4F0900076
:10392700D0E0601474069000B7F074009006E8F0D9
:1039370074009006E9F0800C74009000B7F07406EC
:103947009006E8F09000D0E0B4021474079000B835
:10395700F074009006ECF074009006EDF0800C74A3
:10396700009000B8F074079006ECF09000FCE0B40B
:103977000114741B900122F074009006F4F0740097
:103987009006F5F0800C7400900122F0741B9006ED
:10399700F4F0D2309000D0E0900092F09000FCE07C
:1039A700900093F09000EEE0900094F09000A3E078
:1039B700900095F09000A3E090007AF09000FCE072
:1039C70090007FF09000D0E0900080F09000EEE053
:1039D700900081F0900106E0B4011790002B740F5E
:1039E700F0A374FFF090002DE4F0A3F074029001AF
:1039F70006F0900106E0B4034190002DE0FEA3E03D
:103A0700FF90002BE0FCA3E0FD126B917410126B8A
:103A1700457408120039EF90008BF0EF700674FFC1
:103A270090008BF07400900106F090002CE090005D
:103A37008CF090002BE090008DF0900097E09000C4
:103A470053F0900053E0240C900054F0900053E0A2
:103A57002418900055F0900053E02424900056F06D
:103A6700900053E02430900057F0900054E0D39436
:103A77003C400B900054E0C3943C900054F09000FD
:103A870055E0D3943C400B900055E0C3943C900024
:103A970055F0900056E0D3943C400B900056E0C39D
:103AA700943C900056F0900057E0D3943C400B9024
:103AB7000057E0C3943C900057F090005DE4F0900D
:103AC7000053E0643B6007900053E0B43C20900053
:103AD70053E0B43B06740290005DF0900053E0B4ED
:103AE7003C0690005D7401F09000537401F0900063
:103AF7005EE4F0900054E0643B6007900054E0B44B
:103B07003C20900054E0B43B06740290005EF090B5
:103B17000054E0B43C0690005E7401F090005474C9
:103B270001F090005FE4F0900055E0643B6007907F
:103B37000055E0B43C20900055E0B43B0674029079
:103B4700005FF0900055E0B43C0690005F7401F010
:103B57009000557401F0900060E4F0900056E06426
:103B67003B6007900056E0B43C20900056E0B43B21
:103B7700067402900060F0900056E0B43C06900096
:103B8700607401F09000567401F0900061E4F090C9
:103B97000057E0643B6007900057E0B43C2090007A
:103BA70057E0B43B067402900061F0900057E0B410
:103BB7003C069000617401F09000577401F090008A
:103BC70097E0FE9000FAE02E900063F09000D5E0B9
:103BD700B40173900063E075F00C84AFF07E00EFE2
:103BE7004E7006900063E004F0900063E00475F007
:103BF7000C84AFF07E00EF4E7006900063E014F087
:103C0700900058E0B43D069000587401F0900063AE
:103C1700E0D3943C400B900063E0C3943C90006376
:103C2700F0900063E0D3941E400D900063E0C394CE
:103C37001E900064F0800A900063E0241E900064E8
:103C4700F075511E8041900063E075F00C84AFF071
:103C57007E00EF4E7006900063E004F0900063E092
:103C67000475F00C84AFF07E00EF4E700690006391
:103C7700E014F0900063E075F00C84AFF07E00EF85
:103C8700900063F075510C9000DEE0B402028003EF
:103C9700023D799000DDE0D3943C400D9000DDE0DB
:103CA700C3943C9000DDF0D2309000DDE0900058E6
:103CB700F0900058E075F00C84AFF07E00EF4E7086
:103CC70006900058E004F0900058E00475F00C846A
:103CD700AFF07E00EF4E7006900058E014F09000B1
:103CE70058E0B43D069000587401F0900058E02465
:103CF7000C900059F0900058E0241890005AF0906A
:103D07000058E0242490005BF0900058E0243090A5
:103D1700005CF0900059E0D3943C400B900059E0D0
:103D2700C3943C900059F090005AE0D3943C400B68
:103D370090005AE0C3943C90005AF090005BE0D3A7
:103D4700943C400B90005BE0C3943C90005BF09088
:103D5700005CE0D3943C400B90005CE0C3943C9043
:103D6700005CF0C226C227C228C229C22AD22B026F
:103D77003E9D9000DDE0900058F0900058E075F00F
:103D87000C84AFF07E00EF4E7006900058E004F010
:103D9700900058E00475F00C84AFF07E00EF4E7091
:103DA70006900058E014F0900058E0B479069000AF
:103DB700587401F0900058E0D3943C400F9000589D
:103DC700E0C3943C900058F0D2268002C2269000AF
:103DD70058E02418900059F0900058E024309000E3
:103DE7005AF0900058E0244890005BF0900058E0AB
:103DF700246090005CF0A2269227A2269228A22691
:103E07009229A226922A900059E0D3943C40109020
:103E17000059E0C3943C900059F0A226B392279032
:103E2700005AE0D3943C401090005AE0C3943C9071
:103E3700005AF0A226B3922890005BE0D3943C404E
:103E47002690005BE0D39478400D90005BE0C3942C
:103E57007890005BF0801090005BE0C3943C90008A
:103E67005BF0A226B3922990005CE0D3943C4026F5
:103E770090005CE0D39478400D90005CE0C39478A8
:103E870090005CF0801090005CE0C3943C90005C74
:103E9700F0A226B3922A22C293C294C291C292C2BE
:103EA70087C290E5B554EFF5B5E5B554DFF5B5C272
:103EB70096C295C2A0C297C2A2C2A1E5B554BFF5EA
:103EC700B5E5B5547FF5B5E5B554FBF5B5C2107545
:103ED7005E469000E0E07005756D028003756D0326
:103EE70075550075540090001474FFF0A374DCF04E
:103EF700C218C21AC21CC21EC22074C890003FF06A
:103F070074C8900043F074C8900047F074C89000DC
:103F17004BF074C890004FF0755300755200C20BF8
:103F2700754700E56FB40903756F0075630090006E
:103F370021E4F0A3F0757010C213C214C215C216A3
:103F4700C2179007D0E0FEA3E0FF7403126B45741D
:103F5700011200399007CEEEF0A3EFF0C2027557B9
:103F670000755600900018E4F0A3F0C231755900AF
:103F77007558009000A2E075F032A4FDACF09000F7
:103F870029ECF0A3EDF0C2412275A71085F97385DE
:103F9700FA747E017F00E574126B45E5732FFF50BD
:103FA700010E8E5A8F5BAC5CAD5DEF2DFDEE3CFCD8
:103FB7008C5C8D5D12366A12367512368012368B1E
:103FC70012369675A7002285F97385FA747E017FEC
:103FD70000E574126B45E5732FFF50010E8E5A8F63
:103FE7005B7E017F7690011BE0126B45AC5AAD5B9F
:103FF700ED2FFFEC3EFE8E5C8F5DE55DF5EDE55C3C
:10400700F5EE90008FE4F07412900066F02285F9C7
:104017007385FA747E017F00E574126B45E5732F93
:10402700FF50010E8E5A8F5B9007D0E0FCA3E0FD96
:10403700EF2DFDEE3CFC8C5C8D5DE55DF5FDE55CF3
:10404700F5FE22056422A2DBB340089000EAE09067
:10405700008FF0A2DCB3400AC296C295C2A0C297F5
:10406700C2A275D8402285A77275A710A2D8B340FF
:1040770002C293A2D9B34002C294A2DAB34002C2E9
:1040870091A2DBB34002C292A2DCB34002C28775A1
:10409700D8408572A722900047E4936406600280A7
:1040A700FE74C89007D6F8E4F0E8A3F075B500757C
:1040B700840175A70075FFA0900062E4F075C91030
:1040C70075A70F75A1C775A70075D90075CE0C75B3
:1040D700A70F75F1FE75F2FF75F30775F47875A4F0
:1040E700BA75A5FF75A60775AE0075AFFF75D481C4
:1040F70075D5FF75D6FF75D7FF75A70075A2017532
:10410700A14775F80975D80075D90475DD0975DEFD
:104117000975D84075A71075D80075D90475DA09DF
:1041270075DB0975DC0975DD0975DE0975D840751C
:10413700A70075E60875E71075BC0175BE0475BD67
:104147006C75BE0775BDA075BE0875BD0175BC0051
:1041570075BB1875BC2075BA0875E88075D11375DD
:10416700A70F75E10575E20075C740123E9E75976A
:1041770000759780740A126B257597C0E5975420D0
:10418700700280F8758F0275A700D2AF7598007519
:10419700A90C75A70F75AB4375ADFB75AC1E75A75D
:1041A7001075C91875CA0075CB0075C80475A700C6
:1041B700758912758E04758C00758A00C2A9D28C18
:1041C700758D00758B00D2ABD28E75EF0675D9440D
:1041D700C29974C8F5097508001200E375B5001295
:1041E70004E374639007D6F8E4F0E8A3F012036FD2
:1041F70074C89007D6F8E4F0E8A3F07464F509757D
:1042070008001200E390007AE09000A3F0C2249027
:1042170000A3E0D39403400674009000A3F090003D
:10422700A3E0906394F82828738028A2B44002D2B0
:1042370024802075A70F75F30F75A700A2A340026E
:10424700D224800F75A70F75F31775A700A2A44096
:0342570002D2246C
:0C63940002423002423202423A02424B06
:10425A00A224B34066757308E573D3940E5020E523
:10426A00739007D6F8E4F0E8A3F012023E7464F5FE
:10427A00097508001200E37873740126F650D974A0
:10428A00029000DFF09000A3E0D39403400674008C
:10429A009000A3F09000A3E09063A0F82828738010
:1042AA00167400900109F0800E74009000EEF08000
:0742BA000674009000FBF008
:0C63A0000242A90242AB0242B30242BB1F
:1042C100D2238064757301E573D394075020E5739D
:1042D1009007D6F8E4F0E8A3F012023E7464F50901
:1042E1007508001200E37873740126F650D9740141
:1042F1009000DFF09000A3E0D39403400674009097
:1043010000A3F09000A3E09063ACF8282873801616
:104311007400900109F0800E74009000EEF08006A8
:0643210074009000FBF0A7
:0C63AC0002430F02431102431902432177
:10432700C223900079E0900134F090007AE0900089
:10433700A3F090007BE09000C3F090007CE0900039
:10434700ECF090007DE0900098F090007EE0900007
:10435700DEF090007FE09000FCF0900080E090009D
:10436700D0F0900081E09000EEF0900082E09001A4
:104377001EF09000E9E07006740A9000E9F09000E2
:10438700CAE0700674E39000CAF09000D0E0049091
:104397000092F0123738E5B54401F5B57406900080
:1043A70068F07401900069F0740390006BF0740575
:1043B70090006CF0741D90006DF0740590006EF025
:1043C70090006AE0B40406740490006EF0740090E4
:1043D700006FF07400900074F07400900075F07432
:1043E70001900076F07400900077F074FF900078E9
:1043F700F0743690016DF0743090016EF0742D906A
:10440700016FF07432900170F07420900171F074B4
:1044170035900172F07443900173F07479900174D0
:10442700F0746C900175F07420900176F074209010
:104437000177F07420900178F07420900179F0747E
:104447002090017AF0742090017BF0900105E090B4
:10445700008BF09000BCE090008CF09000BDE090E5
:10446700008DF0A2B6B3920CA2B3B3920DA2A4B37F
:10447700922DA2B4B3922EA2A3B3922F900087E4F9
:10448700F0756F00743A900796F074FD900797F0F7
:10449700900088E4F09007D0E0FEA3E0FF740312D9
:1044A7006B4574011200399007CEEEF0A3EFF0755B
:1044B7006E01900066E4F0C22C756300C211D2123F
:1044C700C202757100C233D203C234D204C235D2DC
:1044D70005C236D206C237D207C238D208C239D28D
:1044E70009C23AD20AC225C22BC23012009E755F9A
:1044F70000756B007561007565327566007567003C
:10450700756800756900756A00900021E4F0A3F0F2
:10451700756C00D2B2D2A4D2B0D2B1D2A3D2A7D2F4
:10452700A6D2A5D2B79000A2E0D394FA400674FAB7
:104537009000A2F07E017F0090008DE0126B459005
:10454700008CE02FFF50010E90002BEEF0A3EFF050
:10455700EFD394FFEE940F400790002BE4F0A3F005
:1045670090008BE0700674FF90008BF07400900051
:10457700C9F09000DFE0D39402400674019000DF99
:10458700F09000E0E07005756D028003756D039093
:1045970000E1E0D39401400674009000E1F0900040
:1045A700E7E0C3940A5006740A9000E7F09000F120
:1045B700E0700674019000F1F09000F1E0B4FF069E
:1045C70074FE9000F1F09000F8E0D394FE4006747A
:1045D700FE9000F8F090011EE0D3940240067401AB
:1045E70090011EF0900134E0D394014006740190CD
:1045F7000134F074019000FEF074019000FFF07434
:1046070000900106F07400900126F074299006DCF2
:10461700F0742A9006E0F074089006F0F0741C908D
:1046270006F8F0D29C9000D1E0D3940440067404BD
:104637009000D1F0900103E0D394044006740490F5
:104647000103F0E570D3941040037570109006DDF8
:10465700E0D3940C400674009006DDF09006E1E08C
:10466700D3940C400674009006E1F09006E5E0D381
:10467700940C400674009006E5F09006E9E0D394A8
:104687000C400674009006E9F09006EDE0D3940C18
:10469700400674009006EDF09006F1E0D3940C40CC
:1046A7000674009006F1F09006F5E0D3940C4006EE
:1046B70074009006F5F09006F9E0D3940C40067468
:1046C700009006F9F0D2EC75CF01A298B34005C26D
:1046D70098120616E54E6006A299B3B3400280050C
:1046E700C299120AB4E54F64016005E54FB40402AC
:1046F70080D5C28E7E107F00E564126B45E58D750F
:10470700F010A4FDACF0EF2DFDEE3CFCE58B75F051
:104717001084FF7E00ED2FFFEC3EFE8E548F55D2A6
:104727008E9000C3E060099000C3E0C3943D40024F
:104737008056900023126B53900023E0FEA3E0FF06
:10474700900025E0FCA3E0FDEFB5053CEEB504388D
:10475700B222A20BB34013A222B34008E5B544042A
:10476700F5B58006E5B554FBF5B5900025E0FEA349
:10477700E0FF900027E0FCA3E0FDEF2DFDEE3CFC01
:10478700900025ECF0A3EDF09000D0E060099000D8
:10479700D0E0C394034002807D1229C0A20BB3501E
:1047A70009900087E0C3942B400280069000BAE08E
:1047B700F546E54675F005A4FFAEF09007D8EEF094
:1047C700A3EFF09000A7E0C395614007E55FC395AD
:1047D7006050079007D8E4F0A3F0AE2FAF309007F2
:1047E700D8E0FCA3E0FDEFD39DEE9C4004C290808F
:1047F7000B900087E0C394415002D2909000D0E024
:10480700B40213A290B34008E5B554EFF5B580069E
:10481700E5B54410F5B59000D0E0B4031C122ADBCF
:10482700AE2FAF309007D8E0FCA3E0FDEFD39DEEAD
:104837009C4004D2908002C2909000ABE06009A235
:10484700B3300D01B3B340028039A2B3300D01B3C9
:104857004031A2B3300F01B3401C9000DEE0B40337
:1048670006A225B3B3400280067404900066F0D216
:1048770025A20FB3920DA20FB330B301B34004A228
:104887000F920DA2B6300C01B35003024F28A2B607
:10489700300C01B35003024F28A2B6300E01B350BB
:1048A70003024D88756E009000C3E0B43D13A20E5D
:1048B700B34008E5B554FBF5B58006E5B54404F506
:1048C700B5055EA210B3B35013AE54AF55900014A4
:1048D700E0FCA3E0FDEDC39FEC9E4003024A40E5E8
:1048E7006DB4032EA231B34022E55EB43B03756D70
:1048F70001E55EC3943B50069000667401F0E55EE7
:10490700D3943B40067402900066F0755E01D23185
:104917008060E56DB40206756D01755E3BE55EB4BA
:104927003B05755E01804B900066E07036E55EC31F
:10493700943B50069000667401F0E55ED3943B40CB
:10494700067402900066F0E55EC3943B5002D22CD9
:10495700E55ED3943B4002D22CC296C295C2A0C258
:1049670097C2A29000E0E0B40105123E9E80037555
:104977005E01AE56AF57AC54AD55EF2DFDEE3CFC86
:1049870074028C068D071200398E568F579000C31C
:10499700E060099000C3E0C3943D4002804390006B
:1049A70023E0FEA3E0FF9000C3E08E048F05FF1213
:1049B7006B3574018C068D07120039900027EEF0D5
:1049C700A3EFF0900027E0F8A3E0900025C8F0A33C
:1049D700C8F0900023E4F0A3F0C222E5B554FBF53C
:1049E700B5A2B4B34002C22EA2A4B34002C22DA204
:1049F700A3B34002C22FA22CB34002C22C9000DE08
:104A0700E0B40331A225B34006A226922B8002B25E
:104A17002B9000ABE06012E56D700EA225B3500934
:104A2700A22B302601B3B3400280067405900066BE
:104A3700F0C2258002D22B803AAE56AF57AC54ADA8
:104A470055EF2DFDEE3CFC74018C068D07120039E5
:104A57008E568F57E56DC39402500DAC54AD557407
:104A6700B8C39D740B9C40028009123E9E74069049
:104A77000066F0E55EB43B127403900066F0D22C3A
:104A87009000E0E0B40103123E9EAE58AF59AC541B
:104A9700AD55EF2DFDEE3CFC8C588D59AE54AF55FE
:104AA700EFD39DEE9C401190001BE0FAA3E0FBEBD7
:104AB700C394E8EA94034002800690001B126B53EC
:104AC700900018E0FEA3E0FFAC54AD55EF2DFDEECE
:104AD7003CFC900018ECF0A3EDF09000E0E0B4018E
:104AE70018AE54AF557405126B4574011200399016
:104AF7000014EEF0A3EFF08011AE54AF557402121C
:104B07006B45900014EEF0A3EFF0C28E758D007523
:104B17008B00756400755501755400D28EE55E24CF
:104B27000E75F00F84AFF07E00EF4E707590001891
:104B3700E0F8A3E0900016C8F0A3C8F0900016E0D4
:104B4700FEA3E0FFEF4E600B7C7D7D69126A338E1A
:104B5700528F53900018E4F0A3F0AE52AF5374286D
:104B6700BE00039F5010E5632FFF50010E74011222
:104B770000398E528F538553639000E7E0A852B8EF
:104B8700000DD395534008E553900065F0800990D8
:104B970000E7E014900065F0E56D60067553007559
:104BA7005200E55E640B6005E55EB429099000D00C
:104BB700E0600312202B9000D5E0B401149000634D
:104BC700E0655E6007900064E0B55E03756F008086
:104BD7001E900063E0655E6013900063E024186533
:104BE7005E6009900063E02424B55E03756F00A240
:104BF70011B35006A210B3B34003024CA990009C16
:104C0700E0B4017390011EE0B40214120C55900039
:104C170090E075F0BEA4FFAEF08E5C8F5D8056E528
:104C27006775F00A84FF7E00900596126B6CE0F5BD
:104C37005B755A00AE5AAF5B9000C1E0126B4574CA
:104C4700648E048F05FF126B358C5C8D5DE55D907E
:104C5700001AF0AE5AAF5B90009AE0126B4574648D
:104C67008E048F05FF126B3574BE8C068D07126B91
:104C7700458E5C8F5D801790009AE075F0BEA4FFAB
:104C8700AEF08E5C8F5D9000C1E090001AF0E56198
:104C9700C394CC500690009AE070028003123F90B4
:104CA700D211E56DB40106E55E64116002800975F5
:104CB70070019000677401F0E56D6003024D839009
:104CC70000E3E0600D90008FE0A852B8000695530E
:104CD700400280509000E3E0B4022F900053E0655B
:104CE7005E601F900054E0655E6017900055E065B8
:104CF7005E600F900056E0655E6007900057E0B574
:104D07005E03757003756C00800CC200756C0090B3
:104D17000021E4F0A3F090008FE060067409900092
:104D270066F08058900053E0B55E0B7570019000F7
:104D3700677401F08046900054E0B55E0B75700112
:104D47007402900067F08034900055E0B55E0B75F3
:104D570070017403900067F08022900056E0B55E02
:104D67000B7570017404900067F08010900057E095
:104D7700B55E097570017405900067F0A20EB392D5
:104D87000CA20EB330B601B35003024F28756E0163
:104D97009000C3E0B43D13A20EB34008E5B5440448
:104DA700F5B58006E5B554FBF5B5E5B54401F5B5B0
:104DB700742B900087F0A20E920CE55ED3944A40C4
:104DC70014D210E55ED39485400B7404900066F00E
:104DD700D22C755E469000EBE0B40107E56AC394F8
:104DE7001440028009123E9E7413900066F0A233AD
:104DF700300301B35017A233B34008E5B54408F5B3
:104E0700B58006E5B554F7F5B5A2339203A2343061
:104E17000401B35017A234B34008E5B54402F5B511
:104E27008006E5B554FDF5B5A2349204A2353005E8
:104E370001B3500FA235B34004D2A18002C2A1A290
:104E4700359205A236300601B3500FA236B340049F
:104E5700D2908002C290A2369206A237300701B3E1
:104E67005017A237B34008E5B54410F5B58006E5FD
:104E7700B554EFF5B5A2379207A238300801B35001
:104E870017A238B34008E5B54420F5B58006E5B567
:104E970054DFF5B5A2389208A239300901B350178B
:104EA700A239B34008E5B54440F5B58006E5B554E9
:104EB700BFF5B5A2399209A23A300A01B35017A239
:104EC7003AB34008E5B54480F5B58006E5B5547FAB
:104ED700F5B5A23A920AE56AC394415009740E9057
:104EE7000066F0123E9E90006EE0FE90006AE004BD
:104EF700C39E400990006AE0D39406400974FB9072
:104F07000066F0123E9E900073E06015900073E01B
:104F1700FE90006DE06E600974FE900066F0123E30
:104F27009EA22CB3400AC296C295C2A0C297C2A243
:104F370090011BE0600CAE52AF537414BE00059F86
:104F4700400280489000A3E09063B8F82828738057
:104F57003BA2B4B35005A22EB340028005123FCE48
:104F6700D22E8028A2A3B35005A22FB340028005FA
:104F7700123FCED22F8015A2A4B35005A22DB34065
:0C4F8700028005123FCED22D8002800077
:1063B800024F56024F58024F6B024F7E024F910216
:0263C8004F93F1
:104F9300A213B3B35008900058E0655E60028044EA
:104FA300A226302B01B340028030A201B35006A2E7
:104FB30000B3B34002802312363A12366A9000FCE3
:104FC300E0B40113A202B34008E5B54440F5B5804F
:104FD30006E5B554BFF5B575A700C213D214D215B3
:104FE300D216D217A214B3B35008900059E0655EED
:104FF30060028044A227302B01B340028030A2011B
:10500300B35006A200B3B34002802312363A1236DD
:10501300759000FCE0B40113A202B34008E5B54467
:1050230040F5B58006E5B554BFF5B575A700D213B5
:10503300C214D215D216D217A215B3B350089000DA
:105043005AE0655E60028044A228302B01B340021F
:105053008030A201B35006A200B3B34002802312F2
:10506300363A1236809000FCE0B40113A202B3403A
:1050730008E5B54440F5B58006E5B554BFF5B5750B
:10508300A700D213D214C215D216D217A216B3B3E5
:10509300500890005BE0655E60028044A229302BDB
:1050A30001B340028030A201B35006A200B3B34063
:1050B30002802312363A12368B9000FCE0B40113BF
:1050C300A202B34008E5B54440F5B58006E5B55402
:1050D300BFF5B575A700D213D214D215C216D217D5
:1050E300A217B3B3500890005CE0655E6002804491
:1050F300A22A302B01B340028030A201B35006A292
:1051030000B3B34002802312363A1236969000FC65
:10511300E0B40113A202B34008E5B54440F5B580FD
:1051230006E5B554BFF5B575A700D213D214D21551
:10513300D216C217E5709063CAF828287302582C58
:04514300900103E0F4
:0663CA00025140025143A4
:105147009063FDF8282873121B078012121B078033
:0E5157000D121B918008121C3D8003121C3D9E
:0F63FD0002514E02515302515802515D0251623A
:1051650075700202582C121D69121E80A241B340AF
:10517500229000C5E0F56C900096E0256CFE90004D
:1051850065E075F01E84FC7F00EE2CF535741090FB
:105195000066F09007CEE0FEA3E0FF740A126B45AF
:1051A500900016E0FCA3E0FD74098F02FF126B3539
:1051B5008D078C038E048A058B06126A339007D2FD
:1051C500EEF0A3EFF09000ECE0B401087430BE00FF
:1051D500059F4002800D74309007D2F8E4F0E8A3F3
:1051E500F0801B9007D2E0FEA3E0FF74F0BE000341
:1051F5009F500B74F09007D2F8E4F0E8A3F0E53582
:1052050070037535019007D2E0FEA3E0FFE5352F69
:10521500FF50010E9007D2EEF0A3EFF075700390EA
:035225000067E03F
:0363D00002516B0C
:1052280090640CF8282873802BA242400375700AFA
:105238008022A242400375700B8019A24240037578
:10524800700C8010A242400375700D8007A2424086
:045258000375700E5C
:10640C0002522F02523102523A02524302524C02B1
:02641C005255D7
:10525C0002582C9006DDE0600312211490011CE032
:10526C00B4011490011DE0A852B8000495535007E6
:10527C00E55FC39560400280030253099000D1E0C2
:10528C00D39402403F9000A5E02403A852B8000438
:10529C00955350099000A7E0D3956150028008D235
:1052AC00017408900066F09000A5E0A852B80005C3
:1052BC00D39553500B9000A7E02403C39561500283
:1052CC00C20180399000A5E02403A852B8000495CF
:1052DC00535007E55FC3956040028008D201740803
:1052EC00900066F09000A5E0A852B80005D3955345
:1052FC005009E560240FC3955F5002C2019000EB8A
:10530C00E07007E56AC3941440028002D201A20146
:10531C004005757004800A757010900021E4F0A3AC
:10532C00F0A20BB34029E56775F00A84FF7E00906C
:10533C000596126B6CE0C394695005122060800FC7
:10534C009007D0E0F8A3E09007CEC8F0A3C8F00215
:06535C00582C9000D1E086
:0663D30002525F02535E5E
:1053620090641EF8282873120D3F8012120D3F80A0
:0E5372000D120EED8008120F9F8003120F9F88
:0F641E0002536902536E02537302537802537D87
:105380009006E1E060031221F075700502582C12BE
:1053900010AB7570069006E5E060031222E09006FF
:1053A000E9E060031223BC02582C90001AE060066A
:1053B000A20BB3B34002801D90001AE0252AFFAE75
:1053C0002950010E8E298F2AE55ED3941450069041
:1053D000001AE014F01212F17570079006EDE0600B
:1053E000031224989006F1E0600312257402582CF1
:1053F00090011EE0B40203120CCD12154E75700818
:105400009006F5E060031226509006F9E060031262
:10541000272C02582C12190A9000DEE0B40305A2D2
:105420000BB34002801590001FE0FEA3E0FF740262
:10543000126B4590001FEEF0A3EFF0A213B35005DE
:10544000A214B34002800AD213D214D215D216D2BB
:105450001775701002582C02582C900041E0C3942C
:10546000465008C2967446900041F090005DE0B44A
:10547000011DE5352406F5359007D2E0FEA3E0FFD7
:1054800074062FFF50010E9007D2EEF0A3EFF090BC
:10549000005DE0B4021DE535240CF5359007D2E03F
:1054A000FEA3E0FF740C2FFF50010E9007D2EEF028
:1054B000A3EFF085355B755A00900053E0F5731249
:1054C00036A1E55D900041F090000AE55AF0A3E5B1
:1054D0005BF0E573900042F0C2199007D2E0F55AF4
:1054E000A3E0F55B900053E0F5731236A1E55D9003
:1054F000003FF0900000E55AF0A3E55BF0E5739003
:105500000040F0C218E56DB4010575700B8003759D
:10551000700302582C900045E0C39446501390004D
:10552000ECE0B40104C2968002C295744690004536
:10553000F090005EE0B4011DE5352406F5359007D6
:10554000D2E0FEA3E0FF74062FFF50010E9007D2B9
:10555000EEF0A3EFF090005EE0B4021DE535240C00
:10556000F5359007D2E0FEA3E0FF740C2FFF500149
:105570000E9007D2EEF0A3EFF085355B755A0090E0
:105580000054E0F5731236A1E55D900045F09000FF
:105590000CE55AF0A3E55BF0E573900046F0C21B02
:1055A0009007D2E0F55AA3E0F55B900054E0F57364
:1055B0001236A1E55D900043F0900002E55AF0A399
:1055C000E55BF0E573900044F0C21AE56DB40105A7
:1055D00075700C800375700302582C900049E0C36D
:1055E000944650139000ECE0B40104C2968002C2CD
:1055F000A07446900049F090005FE0B4011DE535CD
:105600002406F5359007D2E0FEA3E0FF74062FFFD5
:1056100050010E9007D2EEF0A3EFF090005FE0B4DF
:10562000021DE535240CF5359007D2E0FEA3E0FF1E
:10563000740C2FFF50010E9007D2EEF0A3EFF0850F
:10564000355B755A00900055E0F5731236A1E55DA3
:10565000900049F090000EE55AF0A3E55BF0E57389
:1056600090004AF0C21D9007D2E0F55AA3E0F55B26
:10567000900055E0F5731236A1E55D900047F0907B
:105680000004E55AF0A3E55BF0E573900048F0C232
:105690001CE56DB4010575700D800375700302582B
:1056A0002C90004DE0C3944650139000ECE0B40100
:1056B00004C2968002C297744690004DF09000603C
:1056C000E0B4011DE5352406F5359007D2E0FEA3D0
:1056D000E0FF74062FFF50010E9007D2EEF0A3EF0B
:1056E000F0900060E0B4021DE535240CF53590071C
:1056F000D2E0FEA3E0FF740C2FFF50010E9007D202
:10570000EEF0A3EFF085355B755A00900056E0F59A
:10571000731236A1E55D90004DF0900010E55AF04F
:10572000A3E55BF0E57390004EF0C21F9007D2E056
:10573000F55AA3E0F55B900056E0F5731236A1E54B
:105740005D90004BF0900006E55AF0A3E55BF0E5B4
:105750007390004CF0C21EE56DB4010575700E80AB
:105760000375700302582C900051E0C39446501307
:105770009000ECE0B40104C2968002C2A27446908C
:105780000051F0900061E0B4011DE5352406F535C7
:105790009007D2E0FEA3E0FF74062FFF50010E90A9
:1057A00007D2EEF0A3EFF0900061E0B4021DE53502
:1057B000240CF5359007D2E0FEA3E0FF740C2FFF18
:1057C00050010E9007D2EEF0A3EFF085355B755ACD
:1057D00000900057E0F5731236A1E55D900051F09E
:1057E000900012E55AF0A3E55BF0E573900052F0EB
:1057F000C2219007D2E0F55AA3E0F55B900057E094
:10580000F5731236A1E55D90004FF0900008E55A5F
:10581000F0A3E55BF0E573900050F0C220E56DB4B5
:0C5820000103756D0075700380028000AC
:1063D90002538F0253AA0253F00254150254570272
:1063E900545A0255150255DB0256A1025767025845
:0463F9002A02582CF0
:10582C0090003FE0B55E0280030258CEA218407291
:10583C00900000E0FEA3E0FFEF4E6021AE56AF57A4
:10584C00900000E0FCA3E0FD12000374068E048FB0
:10585C0005FF126B35900000ECF0A3EDF0900040CA
:10586C00E0601A900000E0FEA3E0FFAC56AD57EFED
:10587C002DFDEE3CFC900000ECF0A3EDF090004010
:10588C00E0D39401401A900000E0FEA3E0FFAC5678
:10589C00AD57EF2DFDEE3CFC900000ECF0A3EDF0CD
:1058AC00D218AE54AF55900000E0FCA3E0FDEFC35E
:1058BC009DEE9C400D124015D296C21874C89000F3
:1058CC003FF0A218B3B3500790003FE0B55E0280E2
:1058DC000D124015D29674C890003FF0C21890007B
:1058EC0041E0B55E028003025989A2194072900012
:1058FC000AE0FEA3E0FFEF4E6021AE56AF579000DA
:10590C000AE0FCA3E0FD12000374068E048F05FF71
:10591C00126B3590000AECF0A3EDF0900042E060C1
:10592C001A90000AE0FEA3E0FFAC56AD57EF2DFD38
:10593C00EE3CFC90000AECF0A3EDF0900042E0D3BA
:10594C009401401A90000AE0FEA3E0FFAC56AD575C
:10595C00EF2DFDEE3CFC90000AECF0A3EDF0D2191B
:10596C00AE54AF5590000AE0FCA3E0FDEFC39DEEF2
:10597C009C400AC2967446900041F0C219A219B319
:10598C00B35007900041E0B55E02800AC29674469F
:10599C00900041F0C219900043E0B55E0280030212
:1059AC005A4FA21A4072900002E0FEA3E0FFEF4EA5
:1059BC006021AE56AF57900002E0FCA3E0FD120050
:1059CC000374068E048F05FF126B35900002ECF009
:1059DC00A3EDF0900044E0601A900002E0FEA3E01A
:1059EC00FFAC56AD57EF2DFDEE3CFC900002ECF0F9
:1059FC00A3EDF0900044E0D39401401A900002E033
:105A0C00FEA3E0FFAC56AD57EF2DFDEE3CFC900035
:105A1C0002ECF0A3EDF0D21AAE54AF55900002E0B8
:105A2C00FCA3E0FDEFC39DEE9C40181240159000C6
:105A3C00ECE0B40104D2968002D295C21A74C890DC
:105A4C000043F0A21AB3B35007900043E0B55E02D6
:105A5C0080181240159000ECE0B40104D29680023C
:105A6C00D29574C8900043F0C21A900045E0B55E20
:105A7C00028003025B20A21B407290000CE0FEA38C
:105A8C00E0FFEF4E6021AE56AF5790000CE0FCA348
:105A9C00E0FD12000374068E048F05FF126B359027
:105AAC00000CECF0A3EDF0900046E0601A90000CB6
:105ABC00E0FEA3E0FFAC56AD57EF2DFDEE3CFC90A5
:105ACC00000CECF0A3EDF0900046E0D39401401AEA
:105ADC0090000CE0FEA3E0FFAC56AD57EF2DFDEEB1
:105AEC003CFC90000CECF0A3EDF0D21BAE54AF5587
:105AFC0090000CE0FCA3E0FDEFC39DEE9C401590E4
:105B0C0000ECE0B40104C2968002C2957446900089
:105B1C0045F0C21BA21BB3B35007900045E0B55E25
:105B2C000280159000ECE0B40104C2968002C2958C
:105B3C007446900045F0C21B900047E0B55E0280B1
:105B4C0003025BF1A21C4072900004E0FEA3E0FF94
:105B5C00EF4E6021AE56AF57900004E0FCA3E0FD81
:105B6C0012000374068E048F05FF126B359000042F
:105B7C00ECF0A3EDF0900048E0601A900004E0FE19
:105B8C00A3E0FFAC56AD57EF2DFDEE3CFC900004AE
:105B9C00ECF0A3EDF0900048E0D39401401A900093
:105BAC0004E0FEA3E0FFAC56AD57EF2DFDEE3CFC40
:105BBC00900004ECF0A3EDF0D21CAE54AF55900065
:105BCC0004E0FCA3E0FDEFC39DEE9C4018124015D1
:105BDC009000ECE0B40104D2968002D2A0C21C74F6
:105BEC00C8900047F0A21CB3B35007900047E0B533
:105BFC005E0280181240159000ECE0B40104D296BD
:105C0C008002D2A074C8900047F0C21C900049E0FA
:105C1C00B55E028003025CC2A21D407290000EE0D1
:105C2C00FEA3E0FFEF4E6021AE56AF5790000EE0A2
:105C3C00FCA3E0FD12000374068E048F05FF126BAB
:105C4C003590000EECF0A3EDF090004AE0601A9055
:105C5C00000EE0FEA3E0FFAC56AD57EF2DFDEE3C81
:105C6C00FC90000EECF0A3EDF090004AE0D3940110
:105C7C00401A90000EE0FEA3E0FFAC56AD57EF2D9E
:105C8C00FDEE3CFC90000EECF0A3EDF0D21DAE54FA
:105C9C00AF5590000EE0FCA3E0FDEFC39DEE9C40E1
:105CAC00159000ECE0B40104C2968002C2A07446C8
:105CBC00900049F0C21DA21DB3B35007900049E0FB
:105CCC00B55E0280159000ECE0B40104C29680022F
:105CDC00C2A07446900049F0C21D90004BE0B55E26
:105CEC00028003025D93A21E4072900006E0FEA3A8
:105CFC00E0FFEF4E6021AE56AF57900006E0FCA3DC
:105D0C00E0FD12000374068E048F05FF126B3590B4
:105D1C000006ECF0A3EDF090004CE0601A90000649
:105D2C00E0FEA3E0FFAC56AD57EF2DFDEE3CFC9032
:105D3C000006ECF0A3EDF090004CE0D39401401A77
:105D4C00900006E0FEA3E0FFAC56AD57EF2DFDEE44
:105D5C003CFC900006ECF0A3EDF0D21EAE54AF5517
:105D6C00900006E0FCA3E0FDEFC39DEE9C401812F2
:105D7C0040159000ECE0B40104D2968002D297C298
:105D8C001E74C890004BF0A21EB3B3500790004B8A
:105D9C00E0B55E0280181240159000ECE0B40104EE
:105DAC00D2968002D29774C890004BF0C21E90001D
:105DBC004DE0B55E028003025E64A21F407290004B
:105DCC0010E0FEA3E0FFEF4E6021AE56AF579000FF
:105DDC0010E0FCA3E0FD12000374068E048F05FF97
:105DEC00126B35900010ECF0A3EDF090004EE060DB
:105DFC001A900010E0FEA3E0FFAC56AD57EF2DFD5E
:105E0C00EE3CFC900010ECF0A3EDF090004EE0D3D3
:105E1C009401401A900010E0FEA3E0FFAC56AD5781
:105E2C00EF2DFDEE3CFC900010ECF0A3EDF0D21F3A
:105E3C00AE54AF55900010E0FCA3E0FDEFC39DEE17
:105E4C009C40159000ECE0B40104C2968002C2970D
:105E5C00744690004DF0C21FA21FB3B350079000C0
:105E6C004DE0B55E0280159000ECE0B40104C296E2
:105E7C008002C297744690004DF0C21F90004FE014
:105E8C00B55E028003025F35A2204072900008E0EC
:105E9C00FEA3E0FFEF4E6021AE56AF57900008E036
:105EAC00FCA3E0FD12000374068E048F05FF126B39
:105EBC0035900008ECF0A3EDF0900050E0601A90E3
:105ECC000008E0FEA3E0FFAC56AD57EF2DFDEE3C15
:105EDC00FC900008ECF0A3EDF0900050E0D394019E
:105EEC00401A900008E0FEA3E0FFAC56AD57EF2D32
:105EFC00FDEE3CFC900008ECF0A3EDF0D220AE548B
:105F0C00AF55900008E0FCA3E0FDEFC39DEE9C4074
:105F1C00181240159000ECE0B40104D2968002D225
:105F2C00A2C22074C890004FF0A220B3B3500790C7
:105F3C00004FE0B55E0280181240159000ECE0B402
:105F4C000104D2968002D2A274C890004FF0C220F5
:105F5C00900051E0B55E028003026006A2214072FF
:105F6C00900012E0FEA3E0FFEF4E6021AE56AF575B
:105F7C00900012E0FCA3E0FD12000374068E048F67
:105F8C0005FF126B35900012ECF0A3EDF09000526F
:105F9C00E0601A900012E0FEA3E0FFAC56AD57EFA4
:105FAC002DFDEE3CFC900012ECF0A3EDF0900052B5
:105FBC00E0D39401401A900012E0FEA3E0FFAC562F
:105FCC00AD57EF2DFDEE3CFC900012ECF0A3EDF084
:105FDC00D221AE54AF55900012E0FCA3E0FDEFC30C
:105FEC009DEE9C40159000ECE0B40104C29680023A
:105FFC00C2A27446900051F0C221A221B3B3500743
:10600C00900051E0B55E0280159000ECE0B4010404
:10601C00C2968002C2A27446900051F0C221900038
:10602C00EEE0B402028003026146900089E0D39551
:10603C00665064900089E0F4042566FE9000F1E05F
:10604C008E00F5F0E884FF7E008F73EFC394105040
:10605C000CEF8573F0A4FDACF08D7380037573FFAA
:10606C00900089E0D39573400B900089E0C3957341
:10607C00F571800375710090010CE0D395714006A9
:10608C0090010CE0F57190010DE0C39571500690F4
:10609C00010DE0F5718071900089E0C39566FE906A
:1060AC0000F1E08E00F5F0E884FF7E008F73EFC303
:1060BC009410500CEF8573F0A4FDACF08D7380033D
:1060CC007573FF85735B755A00900089E0255BFF43
:1060DC00AE5A50010E8E5A8F5B74FFBE0009D39FCF
:1060EC004005855B7180037571FF90010CE0D395C1
:1060FC0071400690010CE0F57190010DE0C39571B3
:10610C00500690010DE0F571A20BB3B3500D900049
:10611C008AE0FE9000F9E0D39E5002800A7407904A
:10612C000066F0C2A1801375A710E5CDC395714030
:10613C0004C2A18002D2A175A700E56FC3940950D7
:10614C000AA2EDB34005C2ED122C7AAE54AF5574D1
:10615C0010C39F74279E400C900088E0C3945A4053
:10616C0003026391A210B34009123E9E7406900084
:10617C0066F0A224B34008E5B54404F5B58006E505
:10618C00B554FBF5B5900088E0D394014013A212EE
:10619C00B3500EE561D394334007E561C394CC4012
:1061AC0002802FE5B54401F5B5742B900087F09073
:1061BC00009AE075F0BEA4FFAEF08E5C8F5D7402A9
:1061CC00BE000AD39F4006755D02755C00123F90BD
:1061DC00D212900088E0D394014007E561C3941A71
:1061EC0040028002C2129006DDE06003122114A26C
:1061FC0033300301B35017A233B34008E5B544085C
:10620C00F5B58006E5B554F7F5B5A23392039006C3
:10621C00E1E060031221F0A234300401B35017A264
:10622C0034B34008E5B54402F5B58006E5B554FD38
:10623C00F5B5A23492049006E5E060031222E0A2C8
:10624C0035300501B3500FA235B34004D2A1800202
:10625C00C2A1A23592059006E9E060031223BCA20C
:10626C0036300601B3500FA236B34004D2908002F0
:10627C00C290A23692069006EDE06003122498A21A
:10628C0037300701B35017A237B34008E5B54410B7
:10629C00F5B58006E5B554EFF5B5A2379207900633
:1062AC00F1E06003122574A238300801B35017A234
:1062BC0038B34008E5B54420F5B58006E5B554DFA4
:1062CC00F5B5A23892089006F5E06003122650A2AC
:1062DC0039300901B35017A239B34008E5B5444031
:1062EC00F5B58006E5B554BFF5B5A239920990060F
:1062FC00F9E0600312272CA23A300A01B35017A21E
:10630C003AB34008E5B54480F5B58006E5B5547F51
:10631C00F5B5A23A920A900088E0C3945A5010E561
:10632C006FB40909900088E004F0756F00803BE5BC
:10633C006FB40903756F00755500755400758D00A9
:10634C00758B00756400900087E0C39441500890F1
:10635C000087E004F080067441900087F09000877D
:10636C00E0B44106E5B554FEF5B5900088E0D39451
:10637C00014007E56AC3944140028009740E900005
:08638C0066F0123E9E0246CEAF
:10642D000000010001400160018001A001C001E0F8
:10643D0002000300039603B603D603F4040005001F
:10644D000512052405360548055A056C057E05908F
:10645D0005A805C005DE0600061406280646066ECC
:10646D0006AE00FF013F015F017F019F01BF01DF0C
:10647D0001FF02FF039503B503D503F303FF04FFEB
:10648D0005110523053505470559056B057D058F57
:10649D0005A705BF05DD05F1061306270645066DA3
:1064AD0006AD06ED0FAA0FA50F9F0F9A0F940F8D36
:1064BD000F870F800F780F710F680F600F570F4EFA
:1064CD000F450F3B0F300F250F1A0F0E0F020EF554
:1064DD000EE80EDB0ECC0EBE0EAE0E9F0E8E0E7D9A
:1064ED000E6C0E5A0E470E340E200E0C0DF70DE2EB
:1064FD000DCB0DB50D9D0D850D6D0D540D3A0D206A
:10650D000D050CE90CCE0CB10C940C760C580C3A14
:10651D000C1B0BFB0BDB0BBB0B9A0B790B570B35CA
:10652D000B130AF10ACE0AAB0A870A640A400A1C49
:10653D0009F809D409B0098C09670943091F08FB3B
:10654D0008D608B2088E086A0846082307FF07DC3C
:10655D0007B9079607730751072F070D06EC06CAF3
:10656D0006AA068906690649062A060A05EC05CD1E
:10657D0005B0059205750558053C0520050504EA8D
:10658D0004CF04B5049C0482046904510439042227
:10659D00040B03F403DE03C803B2039D03890375E3
:1065AD000361034D033B03280316030402F202E1CA
:1065BD0002D102C002B002A00291028202730265F2
:1065CD0002570249023C022F02220216020901FD66
:1065DD0001F201E601DB01D001C601BB01B101A74A
:1065ED00019D0194018B01820179017001680160A7
:1065FD00015801500148014101390132012B01259A
:10660D00011E01180111010B010500FF00FA0FA673
:10661D000FA00F990F920F8B0F840F7C0F740F6BC0
:10662D000F620F580F4E0F430F380F2C0F1F0F1205
:10663D000F050EF70EE80ED80EC80EB70EA50E9369
:10664D000E800E6C0E580E420E2C0E150DFD0DE427
:10665D000DCB0DB10D950D790D5D0D3F0D200D017E
:10666D000CE10CC00C9E0C7C0C590C350C100BEA7B
:10667D000BC40B9E0B760B4F0B260AFD0AD40AAAF0
:10668D000A800A550A2A09FF09D409A8097C09506C
:10669D00092508F908CD08A10875084A081E07F351
:1066AD0007C8079D07730749072006F706CE06A6FC
:1066BD00067E06570630060A05E405BF059B0577DD
:1066CD0005540532051004EF04CE04AE048F047199
:1066DD0004530435041903FD03E203C703AD03940A
:1066ED00037B0363034B0334031E030802F302DE33
:1066FD0002CA02B602A30291027F026D025C024C35
:10670D00023C022C021D020E020001F201E401D72F
:10671D0001CA01BE01B101A6019A018F0185017A5D
:10672D0001700166015D0153014A014101390131D9
:10673D000129012101190112010B010400FD00F7CE
:10674D0000F000EA00E400DE00D900D300CE00C95D
:10675D0000C400BF00BA00B500B100AD00A800A490
:10676D0000A0009C009900950091008E008A008782
:08677D0000840081007E007B16
:10009E007548009007DAE4F0A3F075320075310070
:1000AE00754E00754F00C23ED23F74FE9007E4F8C5
:1000BE00E4F0E8A3F074FE9007E6F8E4F0E8A3F0AD
:1000CE00745A9007E8F0745A9007E9F0D240C232A1
:1000DE00C242C23D22750B00750A00AE0AAF0BACD0
:1000EE0008AD09EDC39FEC9E401674FF126B25758B
:1000FE00CF01780B740126F6500418E436F650DB67
:10010E0022900062E0B4AA1C900796E0B43C1590D1
:10011E0007D6E0FEA3E0FFEF4E6009741EBE00049A
:10012E00D39F500302023D755D00755C0075F809A2
:10013E009007D6E0FEA3E0FF74076F4E6006740EC4
:10014E006F4E7006743A900796F09007D6E0FEA3B5
:10015E00E0FF7408BE001ED39F401A7E017F0890F8
:10016E0007D6E0FCA3E0FD1DBDFF011C1200038EAF
:10017E005A8F5B801F9007D6E0FEA3E0FF74081233
:10018E006B898F048E057E017F08CDCCCD120003C6
:10019E008E5A8F5BAE5CAF5D740CD39F74019E5014
:1001AE0003020238A2F9B3407EE55D455C7003752B
:1001BE00A382AE5CAF5D74016F4E700375A300AE8B
:1001CE005CAF5D74026F4E700D9007D7E075F00254
:1001DE00A4FDACF08DA3AE5CAF5D74036F4E7003E7
:1001EE0075A300AE5CAF5D7403BE00039F5013ACED
:1001FE005AAD5BED2FFFEC3EFE900092126B6CE061
:10020E00F5A3AE5CAF5DEFB40B09EEB4010574144B
:10021E00126B25AE5CAF5DEFB40B07EEB401037548
:10022E00F80D785C126B990201A2900062E4F02244
:10023E00755D00755C0075F8099007D6E0FEA3E0C9
:10024E00FF7408BE001ED39F401A7E017F089007E0
:10025E00D6E0FCA3E0FD1DBDFF011C1200038E5A6B
:10026E008F5B801F9007D6E0FEA3E0FF7408126B31
:10027E00898F048E057E017F08CDCCCD1200038EB2
:10028E005A8F5BAE5CAF5D7411D39F74019E5003A9
:10029E0002036EA2F9B3500302036BE55D455C7079
:1002AE000375A3D2AE5CAF5D74016F4E700375A380
:1002BE0000AE5CAF5D74026F4E700D9007D7E075A7
:1002CE00F002A4FDACF08DA3AE5CAF5D74036F4E77
:1002DE00700375A300AE5CAF5D74046F4E70037552
:1002EE00A300AE5CAF5D74056F4E700375A300AED8
:1002FE005CAF5D74066F4E700375A300AE5CAF5DB0
:10030E0074076F4E700375A300AE5CAF5D74086F1B
:10031E004E700375A300AE5CAF5D7408BE00039F04
:10032E005016AC5AAD5BED2FFFEC3EFE90008D12D9
:10033E006B6CE5A3F075A300AE5CAF5DEFB4100976
:10034E00EEB401057414126B25AE5CAF5DEFB41004
:10035E0007EEB4010375F80D785C126B99020291E9
:10036E0022755D00755C0075F809AE5CAF5D7417A3
:10037E00BE0004D39F5003020447A2F9B3500302F8
:10038E000444E55D455C700375A3D2AE5CAF5D744D
:10039E00016F4E700375A300AE5CAF5D74026F4EBD
:1003AE00700D9007D7E075F002A4FDACF08DA3AEF2
:1003BE005CAF5D74036F4E700375A300AE5CAF5DF2
:1003CE0074046F4E700375A300AE5CAF5D74056F61
:1003DE004E700375A300AE5CAF5D74066F4E700376
:1003EE0075A300AE5CAF5D74076F4E700375A3000E
:1003FE00AE5CAF5D74086F4E700375A300AE5CAF5C
:10040E005D7408BE00039F500C900070126B6CE57B
:10041E00A3F075A300AE5CAF5D74166F4E700574DD
:10042E0014126B25AE5CAF5D74166F4E700375F8CB
:10043E000D785C126B9902037822900062E0B4ABE7
:10044E000280030204E2755D00755C0075F809AE6A
:10045E005CAF5D7412BE007CD39F4078A2F9B340AE
:10046E0070E55D455C700375A382AE5CAF5D740193
:10047E006F4E700375A300AE5CAF5D74026F4E706D
:10048E000D9007D7E075F002A4FDACF08DA3AE5C25
:10049E00AF5D74036F4E700375A300AE5CAF5D74F9
:1004AE0003BE00039F5009900075126B6CE0F5A31C
:1004BE00AE5CAF5D74116F4E70057414126B25AE89
:1004CE005CAF5D74116F4E700375F80D785C126B36
:1004DE009902045D229007E1E4F074649007D6F867
:1004EE00E4F0E8A3F012036F74C89007D6F8E4F0B6
:1004FE00E8A3F090007CE0B4371A900079E0900009
:10050E0070F090007AE0900071F090007BE0900027
:10051E0072F080469007E17401F074659007D6F88A
:10052E00E4F0E8A3F012036F74C89007D6F8E4F075
:10053E00E8A3F090007CE0B4371A900079E09000C8
:10054E0070F090007AE0900071F090007BE09000E7
:10055E0072F0800674029007E1F09007E2E4F07406
:10056E00669007D6F8E4F0E8A3F012036F74C89013
:10057E0007D6F8E4F0E8A3F090007BE0B4371290D1
:10058E000079E090006AF090007AE0900073F080BD
:10059E00769007E27401F074679007D6F8E4F0E8FD
:1005AE00A3F012036F74C89007D6F8E4F0E8A3F036
:1005BE0090007BE0B43712900079E090006AF090E2
:1005CE00007AE0900073F0803E74029007E2F074BF
:1005DE00689007D6F8E4F0E8A3F012036F74C890A1
:1005EE0007D6F8E4F0E8A3F090007BE0B437129061
:1005FE000079E090006AF090007AE0900073F0804D
:10060E000674039007E2F022E54F64046006E59954
:10061E0064FF6002802AA23E4004D23E8020E54F55
:10062E00600874E6254F900066F0754F00E54E6049
:10063E000874F0254E900066F0754E00C23E8002A2
:10064E00C23EE54F9033F8F8282873754F00E599B0
:10065E00B4FF03754E01E599B4FE03754E02E5999C
:10066E00B4FD03754E03E599B4FC03754E04E5998C
:10067E00B4FA03754E05E599B4FB06754F01123EAB
:10068E009EE599B4F906754F04123E9EE599D394F2
:10069E00E54007E599C394F04002801685995075A0
:1006AE004F027E017F00E550C394E6126B458E33F8
:1006BE008F349007DAE4F0A3F0E599D394C44007A1
:1006CE00E599C394E640028028859950754F0374CE
:1006DE00E5C39550F534753300AE33AF3490642DC9
:1006EE00126B14E493F87401939007DAC8F0A3C860
:1006FE00F0D299020AB3900079E070429007DAE0E6
:10070E00FEA3E0FF74FFBE00039F5009EFC39446A3
:10071E00EE940640119007DAE0FEA3E0FFEFD394CB
:10072E006DEE940640139007DAE0FEA3E0FF900012
:10073E0096126B6CE599F080038599748011900781
:10074E00DAE0FEA3E0FF900096126B6CE599F09054
:10075E0007DA126B539007DAE0FEA3E0FFEFB40165
:10076E0006EEB40702800302089B900796E0B43CA5
:10077E00028003020885C29C900079E0900134F05B
:10078E0090007AE09000A3F090007BE09000C3F020
:10079E0090007CE09000ECF090007DE0900098F0EE
:1007AE0090007EE09000DEF090007FE09000FCF084
:1007BE00900080E09000D0F0900081E09000EEF08C
:1007CE00900082E090011EF012373890008BE0907E
:1007DE000105F090008CE09000BCF090008DE09050
:1007EE0000BDF074639007D6F8E4F0E8A3F074ABA4
:1007FE00900062F0120448900062E4F0750964758E
:10080E0008001200E3A2234038757301E573D394F8
:10081E0007502CE5739007D6F8E4F0E8A3F074AA1D
:10082E00900062F012010FE573C394075009750929
:10083E00647508001200E37873740126F650CD80BB
:10084E0036757308E573D3940E502CE5739007D666
:10085E00F8E4F0E8A3F074AA900062F012010FE53C
:10086E0073C3940E50097509647508001200E3787D
:10087E0073740126F650CD74C89007D6F8E4F0E8EC
:10088E00A3F0D29C754F00754E007599FB020AB30A
:10089E009007DAE0FEA3E0FFEF4E70068599327501
:1008AE0031009007DAE0FEA3E0FF74016F4E701B7B
:1008BE00AC31AD32AA33AB34ED2BFBEC3AFA8A06EF
:1008CE008B07900096126B6CE599F09007DA126B1D
:1008DE00539007DAE0FEA3E0FF74026F4E7021AC76
:1008EE0031AD3274566D4C7006E55064E660028090
:1008FE0003123E9E123738855099754F00754E0083
:10090E00020AB39007DAE0FEA3E0FF900096126BA6
:10091E006CE599F09007DA126B539007DAE0FEA3BC
:10092E00E0FFAC33AD348F028E038C068D079064DE
:10093E006F126B14E493F9740193FEEAD39EEB9954
:10094E004009855099754F00754E00020AB3900705
:10095E00DAE0FEA3E0FF900096126B6CE599F09042
:10096E0007DA126B539007DAE0FEA3E0FFEFB40054
:10097E0006EEB401028003020AB3900072E075F035
:10098E0002A4FDACF08D73ED900096126B77EDFA2C
:10099E00E0FBEA900099126B77EBFAE0FBEA2BFA98
:1009AE00900072E0B502028003020AA50DED9000E0
:1009BE0096126B77E573FDE0FAED90009A126B7765
:1009CE00EAFDE0FAEDC39AFD900072E0B5050280F3
:1009DE0003020AA5E573900098126B77E573FDE0AC
:1009EE00FAED90009B126B77EAFDE0FAED2AFD908E
:1009FE000072E0B505028003020AA5E57390009C23
:100A0E00126B77FDE0FAED900072E0F4042A90008C
:100A1E0079F0E57390009D126B77FDE0FAED900092
:100A2E0072E0F4042A90007AF0E57390009E126B47
:100A3E0077FDE0FAED900072E0F4042A90007BF06E
:100A4E00E57390009F126B77FDE0FAED900072E077
:100A5E00F4042A9007D6F8E4F0E8A3F074AB900003
:100A6E0062F01204487509647508001200E39007DD
:100A7E00D6126B531204487509647508001200E310
:100A8E009007D6126B531204487599F9750964755F
:100A9E0008001200E380FE7599FF75096475080061
:050AAE001200E380FED0
:0F33F80002065902070402089E02091102095C2D
:100AB30022E54E903407F8282873020B989007DA42
:100AC300E0FEA3E0FF900068126B6CE0F5999007DD
:100AD300DA126B539007DAE0FEA3E0FF74116F4E56
:100AE3007003754E00020B98856E99020B98900760
:100AF300DAE0FEA3E0FF900096126B6CE0F599EF4D
:100B0300B40107EEB40703754E009007DA126B5376
:070B1300020B989007DBE0E4
:0F340700020ABD020AC0020AEB020AF1020B160A
:100B1A009035BAF82828738553998067855F99803C
:100B2A0062856199805D856599805885679980534A
:100B3A00856899804E8569998049856A998044902B
:100B4A000022E0F599803CA23FB340077599FAC2AA
:100B5A003F8017A230B3400575990F800B9000664D
:100B6A00E0F599900066E4F0C2308017856B9980B1
:100B7A0012856699800D856C9980087599FC8003A9
:030B8A00754E00A5
:1035BA00020B21020B26020B2B020B30020B3502E7
:1035CA000B3A020B3F020B44020B49020B51020B4E
:0D35DA0076020B7B020B80020B85020B8A30
:0B0B8D009007DA126B5380031235E76B
:03341600020B9511
:100B980022E538255BFFAE5A50010E900096126B85
:100BA8006CE0F539E538255BFFAE5A50010E0FBFF2
:100BB80000010E900096126B6CE0F53A85403CE51A
:100BC80039B53A058539388041E53AD39539401D1C
:100BD800E53AC39539853BF0A4FFAEF0E53C8E04B9
:100BE8008F05FF126B35ED2539F538801DE539C3C2
:100BF800953A853BF0A4FFAEF0E53C8E048F05FFE7
:100C0800126B35EDF4042539F53822E53AD39539D8
:100C1800401DE53AC39539853BF0A4FFAEF0E53CAD
:100C28008E048F05FF126B35ED2539F538801DE5EB
:100C380039C3953A853BF0A4FFAEF0E53C8E048FAE
:100C480005FF126B35EDF4042539F5382290009C28
:100C5800E0B40170E56775F00A84FF7E008F38E51F
:100C68006775F00A84ADF07C008D3B75400A755AB3
:100C780005755B24E538C394115005120B9980065D
:100C88009005CBE0F538E538900090F0E56775F011
:100C98000A84FF7E008F38E56775F00A84ADF07C22
:100CA800008D3B75400A755A05755B5AE538C39443
:100CB800115005120B998006900601E0F538E538C9
:100CC80090001AF02290009CE0B4016AE56775F084
:100CD8000A84FF7E008F38E56775F00A84ADF07CE2
:100CE800008D3B75400A755A05755B36E538C39427
:100CF800115005120B9980069005DDE0F53885380E
:100D08004CE56775F00A84FF7E008F38E56775F05B
:100D18000A84ADF07C008D3B75400A755A05755BF9
:100D280048E538C394115005120B9980069005EFD9
:100D3800E0F53885384D22E55F75F00484FF7E00C4
:100D48008F38E55F75F00484ADF07C008D3B75400D
:100D580004755A01755B00E538C3943F5005120BC2
:100D68009980069001D5E0F53885382A75290090D4
:100D78000065E075F020A4FFAEF09000E7E08E0477
:100D88008F05FF126B358D389000CFE0D3955F50FB
:100D980003020E459000F3E0D3955F4010ED9001FB
:100DA800D6126B77E0F52C752B00020E429000BE30
:100DB800E0D3955F4043E5389001D6126B77E0F5B4
:100DC80039E5389001F6126B77E0F53A9000F3E0D8
:100DD800F404255FF53B9000BEE0FE9000F3E0F4DC
:100DE800042EF53CE539B53A058539388003120CEF
:100DF8001385382C752B008041E5389001F6126B6D
:100E080077E0F539E538900216126B77E0F53A90FD
:100E180000BEE0F404255FF53B9000CFE0FE9000B3
:100E2800BEE0F4042EF53CE539B53A05853938803D
:100E380003120C1385382C752B00020EEC9000F66B
:100E4800E0D3955F5011E538900256126B77E0F5C4
:100E58002C752B00020EEC9000BFE0D3955F504339
:100E6800E538900236126B77E0F539E5389002568E
:100E7800126B77E0F53A9000BFE0F404255FF53B8C
:100E88009000F6E0FE9000BFE0F4042EF53CE53952
:100E9800B53A058539388003120C1385382C752B23
:100EA800008041E538900216126B77E0F539E53895
:100EB800900236126B77E0F53A9000CFE0F4042503
:100EC8005FF53B9000BFE0FE9000CFE0F4042EF504
:100ED8003CE539B53A058539388003120C13853855
:100EE8002C752B0022900107E0F53D754011755ACD
:100EF80002755B00AE52AF53E53D75F00FA4FDAC33
:100F0800F0EDD39FEC9E4021E53D8E048F05FF1246
:100F18006B35ED75F010A4FFAEF0E55F75F0118448
:100F2800FD7C00ED2FF53E800EE55F75F01184FF26
:100F38007E00EF24F0F53E853E38E55F75F01184BC
:100F4800AFF07E008F3B120B9985383FAE52AF53FE
:100F5800900107E075F00FA4FDACF0EDD39FEC9E77
:100F68004028755A02755B10853E38120B99853FEB
:100F78003985383AAE52AF53E53D8E048F05FF12DE
:100F88006B608D3B853D3C120C1385382A75290012
:100F9800752C64752B0022900107E0F53D75401112
:100FA800755A02755B00AE52AF53E53D75F00FA45C
:100FB800FDACF0EDD39FEC9E4021E53D8E048F05FE
:100FC800FF126B35ED75F010A4FFAEF0E56175F01A
:100FD8001184FD7C00ED2FF53E800EE56175F01162
:100FE80084FF7E00EF24F0F53E853E38E56175F01C
:100FF8001184AFF07E008F3B120B9985383FAE52BB
:10100800AF53900107E075F00FA4FDACF0EDD39F4E
:10101800EC9E4028755A02755B10853E38120B9974
:10102800853F3985383AAE52AF53E53D8E048F057A
:10103800FF126B608D3B853D3C120C1385382A7579
:1010480029009000D1E0B40453E55F75F00484FFF3
:101058007E008F38E55F75F00484ADF07C008D3B31
:10106800754004755A01755B00E538C3943F500517
:10107800120B9980069001D5E0F538AE29AF2AE524
:1010880038126B4574648E048F05FF126B35AE29D8
:10109800AF2AEF2DFDEE3CFC8C298D2A752C64754A
:1010A8002B002290009CE0B40146E56775F00A84A5
:1010B800FF7E008F38E56775F00A84ADF07C008DFF
:1010C8003B75400A755A05755B00E538C3941150A5
:1010D80005120B9980069005A7E0F538AE2BAF2CCA
:1010E800E5382FFF50010E7464126B898E2B8F2CFC
:1010F80090009DE0B40146E56875F00A84FF7E0023
:101108008F38E56875F00A84ADF07C008D3B75403A
:101118000A755A05755B6CE538C394115005120BB6
:10112800998006900613E0F538AE2BAF2CE5382FE2
:10113800FF50010E7464126B898E2B8F2C9000ACBB
:10114800E0B40249E56AC3944175F00584FF7E0066
:101158008F38E56A75F00584ADF07C008D3B7540ED
:1011680005755A06755B00E538C394135005120BD4
:101178009980069006A9E0F538AE2BAF2CE5382FFC
:10118800FF50010E7464126B898E2B8F2C9000EE29
:10119800E0B40202800302124AE55F75F01584FF8D
:1011A8007E008F38E55F75F01584ADF07C008D3BCF
:1011B800754015755A03755BF4E538C3940B5005F3
:1011C800120B998006900495E0F538E53875F0FF24
:1011D800A4FFAEF09000EFE08E048F05FF126B3590
:1011E800ED900089F0E56675F078A4FFAEF074FF25
:1011F8008E048F05FF126B358C5A8D5B74028C063A
:101208008D071200398F38AC5AAD5B7404FF126B2E
:10121800608D3B754004755A06755B28E538C394A4
:101228001D5005120B9980069006DBE0F538AE2BB1
:10123800AF2CE5382FFF50010E7464126B898E2B8A
:101248008F2C90009BE0B4025DE56175F064A4FF0B
:10125800AEF074081200398E5C8F5D74058E048FB1
:1012680005FF126B358D38AE5CAF5D74058E048F4B
:1012780005FF126B608D3B754005755A05755BDE81
:10128800E538C394135005120B998006900687E041
:10129800F538AE2BAF2CE5382FFF50010E746412D1
:1012A8006B898E2B8F2C9000DDE0703C900065E000
:1012B80075F00584FF7E008F38900065E075F005B5
:1012C80084ADF07C008D3B754005755A05755BC093
:1012D800E538C3941D5005120B998006900673E0FB
:1012E800F538E538900091F0229000A4E0B4011799
:1012F8009007DDE0252CFFAE2B50010E9000F8E0A2
:10130800126B898E2B8F2C90011CE0B40114900174
:101318001DE0A852B8000495535007E55FC39560D7
:10132800400280129000C6E0252CFFAE2B50010E23
:101338008E2B8F2C802F9000A4E0B40316A232B31A
:10134800B350109007E0E0C39405A852B800069582
:1013580053400280109000C6E0252CFFAE2B5001B0
:101368000E8E2B8F2C90009EE0B402028003021593
:101378004D9000A1E0602FE567D394464028900087
:101388001BE0FEA3E0FF9000DCE075F003A4FDACD9
:10139800F0EFD39DEE9C400E900100E0A852B800FB
:1013A80005D39553500302154D9000E9E0855FF091
:1013B800A4FFAEF07405126B4574071200398E5AFB
:1013C8008F5B9000A8E0A852B80004955350129083
:1013D80000A9E075F002A4FDACF0EFC39DEE9C40BF
:1013E8000302154DE55F75F00B84FF7E009006261D
:1013F800126B6CFEE0FFEE9000A0E0FEEF8E00881E
:10140800F0A4FFAEF074648E048F05FF126B358C68
:101418005A8D5B900065E075F018A4FFAEF090005F
:10142800E7E08E048F05FF126B358C068D0790065A
:101438003E126B6CAE5AAF5BE0126B4574648E045F
:101448008F05FF126B358C5A8D5BE565A85AB8007D
:1014580077D3955B4072E565C3955BFFE4955AFECB
:101468008E5A8F5B7428BE00039F500C755B2875DD
:101478005A00740D900066F0AE5AAF5B9000A1E080
:10148800126B4574288E048F05FF126B358C5A8DAC
:101498005BAE29AF2A740A8E048F05FF126B358D57
:1014A800068C07AC5AAD5BCFCECF120003740A8E00
:1014B800048F05FF126B358C5A8D5BAE29AF2A124B
:1014C8006B918E298F2A807DE565A85AB80004950E
:1014D8005B5072AE5AAF5BE565126B898E5A8F5BB3
:1014E8007428BE00039F500C755B28755A00740D54
:1014F800900066F0AE5AAF5B9000A1E0126B4574A5
:10150800288E048F05FF126B358C5A8D5BAE29AF80
:101518002A740A8E048F05FF126B358D068C07AC72
:101528005AAD5BCFCECF120003740A8E048F05FF2D
:10153800126B358C5A8D5BAE29AF2AEF2DFDEE3C30
:10154800FC8C298D2A229000FCE0B4026AE55F75C4
:10155800F00884FF7E008F38E55F75F00884ADF0F1
:101568007C008D3B754008755A01755BE0E538C312
:10157800943F5005120B998006900295E0F5388546
:10158800382E752D00AE2DAF2EAC2BAD2C120003CE
:1015980074648E048F05FF126B358C2D8D2E900090
:1015A80099E08C068D07126B4574648E048F05FFD5
:1015B800126B358C2D8D2EAE29AF2AAC2BAD2C128B
:1015C800000374648E048F05FF126B358C298D2AF5
:1015D800900099E08C068D07126B4574648E048F19
:1015E80005FF126B358C298D2AA20B401DAE52AF18
:1015F800537405BE00039F5002D20BE561D394CC0F
:101608004008D2017411900066F09000FBE0B4022B
:10161800089000FDE0640160028035AE29AF2AE53C
:101628006B126B4574E78E048F05FF126B358C299E
:101638008D2A9000FCE0B40217AE2DAF2EE56B1298
:101648006B4574E78E048F05FF126B358C2D8D2E3C
:101658009000BBE05402601B9000B2E0A852B800B2
:1016680012D39553400DA20BB3B35007E561C39451
:101678009A40028028AE36AF379000B0E075F0028D
:10168800A4FDACF0EF2DFDEE3CFC74022DFD5001E5
:101698000CE561BC0007D39D4003754401856137A3
:1016A800753600E544700302179190010EE0C3956A
:1016B80044500302178390011EE0C394025076E55C
:1016C8006775F00A84FF7E00900596126B6CE0F552
:1016D8005B755A00AE5AAF5B9000B1E0126B45746F
:1016E800648E048F05FF126B358C5C8D5D90010E46
:1016F800E004C395448C068D07126B4590010EE0FB
:101708008E048F05FF126B358C5C8D5DAE29AF2A78
:10171800EF2DFDEE3CFC8C298D2A9000FCE0B402F4
:1017280012AE2DAF2EAA5CAB5DEF2BFBEE3AFA8A18
:101738002D8B2E804690010EE004C39544854CF015
:10174800A4FFAEF090010EE08E048F05FF126B35FA
:101758008C5C8D5DAE29AF2AEF2DFDEE3CFC8C290B
:101768008D2A9000FCE0B40212AE2DAF2EAA5CAB1D
:101778005DEF2BFBEE3AFA8A2D8B2E054490010E75
:10178800E0C3954450037544009000BBE0540160E9
:101798001B9000AFE0A852B80012D39553400DA299
:1017A8000BB3B35007E55FC394CC4002802590008B
:1017B800ADE075F003A4FFAEF0E5412FFF50010E38
:1017C80074032FFF50010EE55FBE0007D39F40034F
:1017D800754501855F41E54570030218C490010F06
:1017E800E0C3954550030218B690011EE0C3940269
:1017F8005076E56775F00A84FF7E00900596126BB7
:101808006CE0F55B755A00AE5AAF5B9000AEE01223
:101818006B4574648E048F05FF126B358C5C8D5D8F
:1018280090010FE004C395458C068D07126B459017
:10183800010FE08E048F05FF126B358C5C8D5DAE59
:1018480029AF2AEF2DFDEE3CFC8C298D2A9000FC57
:10185800E0B40212AE2DAF2EAA5CAB5DEF2BFBEE0F
:101868003AFA8A2D8B2E804690010FE004C39545E5
:10187800854DF0A4FFAEF090010FE08E048F05FFB8
:10188800126B358C5C8D5DAE29AF2AEF2DFDEE3CD9
:10189800FC8C298D2A9000FCE0B40212AE2DAF2EEC
:1018A800AA5CAB5DEF2BFBEE3AFA8A2D8B2E054531
:1018B80090010FE0C395455003754500900111E074
:1018C800252AFFAE2950010E8E298F2A9000C0E0EC
:1018D800A829B80004952A50099000C0E0F52A7597
:1018E80029009000FCE0B4020D9000C0E0A82DB8DB
:1018F8000006952E400280099000C0E0F52E752D57
:1019080000229000FCE0B401028003021A15A20B29
:10191800B35003021A139000C7E0B40168AE29AFB0
:101928002AAC52AD53120003743C8E048F05FF128B
:101938006B359000D7E0BC00109D400D9000D9E0B9
:10194800A829B80004952A5002D202AE29AF2AACC1
:1019580052AD53120003743C8E048F05FF126B3591
:101968009000D7E0C3940ABC0015D39D40119000A5
:10197800D9E0C39405A829B80005D3952A50028058
:1019880002C2028068AE29AF2AAC52AD53120003DE
:1019980074788E048F05FF126B359000D7E0BC0079
:1019A800109D400D9000D9E0A829B80004952A5050
:1019B80004D2028038AE29AF2AAC52AD53120003CC
:1019C80074788E048F05FF126B359000D7E0C394AE
:1019D8000ABC0015D39D40119000D9E0C39405A816
:1019E80029B80005D3952A50028002C202A202B388
:1019F8004019AE29AF2A9000D8E0126B4574648E66
:101A0800048F05FF126B358C298D2A8002C202A231
:101A180000B34006A201B3B35009900021E4F0A33B
:101A2800F08024AE29AF2A7400D39F74019E400C25
:101A3800900021E529F0A3E52AF0800B74FF9000BF
:101A480021F8E4F0E8A3F09000DEE0D39402400C23
:101A58009000C9E07006A20BB3B34002801AAE2909
:101A6800AF2A7402126B458E298F2AAE2DAF2E74C1
:101A780002126B458E2D8F2E9000C7E0B4011AAE6E
:101A880029AF2A7402126B458E298F2AAE2DAF2EEC
:101A98007402126B458E2D8F2EAE29AF2A745E12FA
:101AA8006B45740A8E048F05FF126B358C298D2ABD
:101AB8009000FCE0B40217AE2DAF2E745E126B4599
:101AC800740A8E048F05FF126B358C2D8D2EAE296E
:101AD800AF2A7402BE000AD39F4006752A027529F0
:101AE80000AE2DAF2E7402BE000AD39F4006752E9D
:101AF80002752D0090001FE529F0A3E52AF0229039
:101B08000065E0900396126B77E0F54275436490A8
:101B18000065E0FE9000D2E0D39E4037E55F75F0A7
:101B28000884FF7E008F38E55F75F00884ADF07C8F
:101B3800008D3B754008755A03755B96E538C3946C
:101B48001F5005120B99800690044BE0F538853834
:101B5800438035E55F75F00884FF7E008F38E55FC8
:101B680075F00884ADF07C008D3B754008755A030C
:101B7800755BB6E538C3941F5005120B9980069023
:101B8800046BE0F53885384322900108E0F53D758F
:101B98004011755A04755B00AE52AF53E53D75F0C0
:101BA8000FA4FDACF0EDD39FEC9E4021E53D8E04E3
:101BB8008F05FF126B35ED75F010A4FFAEF0E55FF1
:101BC80075F01184FD7C00ED2FF53E800EE55F7504
:101BD800F01184FF7E00EF24F0F53E853E38E55F86
:101BE80075F01184AFF07E008F3B120B9985383F5A
:101BF800AE52AF53900108E075F00FA4FDACF0EDC4
:101C0800D39FEC9E4028755A04755B10853E3812A8
:101C18000B99853F3985383AAE52AF53E53D8E046E
:101C28008F05FF126B608D3B853D3C120C13853888
:101C38004275436422900108E0F53D754011755ADC
:101C480004755B00AE52AF53E53D75F00FA4FDACD3
:101C5800F0EDD39FEC9E4021E53D8E048F05FF12E9
:101C68006B35ED75F010A4FFAEF0E56175F01184E9
:101C7800FD7C00ED2FF53E800EE56175F01184FFC7
:101C88007E00EF24F0F53E853E38E56175F011845D
:101C9800AFF07E008F3B120B9985383FAE52AF53A1
:101CA800900108E075F00FA4FDACF0EDD39FEC9E19
:101CB8004028755A04755B10853E38120B99853F8C
:101CC8003985383AAE52AF53E53D8E048F05FF1281
:101CD8006B608D3B853D3C120C138538427543641F
:101CE800900103E0B40479900065E0FE9000D2E032
:101CF800D39E4037E55F75F00884FF7E008F38E596
:101D08005F75F00884ADF07C008D3B754008755A0E
:101D180003755B96E538C3941F5005120B9980062E
:101D280090044BE0F5388538438035E55F75F00859
:101D380084FF7E008F38E55F75F00884ADF07C0085
:101D48008D3B754008755A03755BB6E538C3941F1B
:101D58005005120B99800690046BE0F538853843DE
:101D68002290009CE0B4013BE56775F00A84FF7E91
:101D7800008F38E56775F00A84ADF07C008D3B75FF
:101D8800400A755A05755B12E538C394115005125F
:101D98000B9980069005B9E0F538E5432538C394DA
:101DA80064F54390009DE0B4013BE56875F00A8452
:101DB800FF7E008F38E56875F00A84ADF07C008DF1
:101DC8003B75400A755A05755B7EE538C39411501A
:101DD80005120B998006900625E0F538E54325386D
:101DE800C39464F543E5422543F5359000A4E0B477
:101DF80002109007DCE02535FE9000F8E0F4042E90
:101E0800F5359000FBE0D394014040E56BC394E7BF
:101E1800501D74E7C3956BFE9007DEE08E00F5F069
:101E2800E884FF7E008F38E5352538F535801CE5D8
:101E38006BC394E7FE9007DEE08E00F5F0E884FFC0
:101E48007E008F38E535C39538F535A20B4006E599
:101E5800422464F535E535D394644009E535C394E7
:101E680064F53580037535009000D4E0C39535508E
:101E7800069000D4E0F53522D20090008FE0A852F9
:101E8800B800049553504190008FE0A852B8000460
:101E98009553500375350F90008FE004A852B80091
:101EA800049553500375350A90008FE02402A85218
:101EB800B8000495535005753505C20090008FE0B1
:101EC80060067409900066F0C2427E017F009000AF
:101ED800DAE0126B459000E9E08E048F05FF126B83
:101EE80035E55FBC0017D39D40139000E3E0B402D2
:101EF80004D2428002C200740A900066F09000DBAF
:101F0800E0C3956750159000EDE0A852B80004951D
:101F1800535002C200740B900066F0E567C39464E6
:101F2800501D900133E0600D900133E0A852B800D5
:101F380006955340028008C200740B900066F0A218
:101F480000400375350590011CE0B4011490011D93
:101F5800E0A852B8000495535007E55FC395604068
:101F68000280089000C5E0F535803A9000A4E0B4FE
:101F78000306A232B3B34002802B9007E0E0C3947B
:101F880005A852B800049553500C9000C5E0F535EB
:101F9800740C900066F09007E0E0A852B800049531
:101FA800535002C20085356C900096E02535FE90AE
:101FB8000065E075F01E84FC7F00EE2CF53522905C
:101FC8000065E075F00584FF7E008F38900065E0BD
:101FD80075F00584ADF07C008D3B754005755A039E
:101FE800755BD69000E7E01475F00584FF7E00E588
:101FF80038BE00039F5005120B99800BE5389004FA
:102008006C126B77E0F538E5389007DFF09007DF62
:10201800E0FE9000D6E0C39E50089000D6E09007FE
:10202800DFF022E56775F00A84FF7E0090059612BE
:102038006B6CE0F547E547D394644010E547C394DB
:102048006475F00F84FF7E008F478003754700900A
:1020580000B9E02547F547229007D0E0FEA3E0FF4E
:102068007404120039E55F126B45740F8E048F05F6
:10207800FF126B359007CEECF0A3EDF09000ACE0CA
:10208800B40262E56AC3944175F00584FF7E008F4F
:1020980038E56A75F00584ADF07C008D3B75400528
:1020A800755A06755B14E538C394175005120B99D9
:1020B80080069006BDE0F5389007CEE0FEA3E0FF6D
:1020C800740A8E048F05FF126B35E5388C068D0770
:1020D800126B45740A8E048F05FF126B359007CE7C
:1020E800ECF0A3EDF09007CEE0FEA3E0FF9007D45C
:1020F800E0FCA3E0FDEDD39FEC9E400F9007D4E0F9
:10210800F8A3E09007CEC8F0A3C8F0229006DDE05F
:10211800903419F8282873804C85537380479000B1
:10212800E9E0855FF0A4FFAEF074081200398F7300
:102138008033856173802E856773802985687380F5
:1021480024856973801F856A73801A856B7380156F
:102158008566738010856573800B856C7380069027
:052168000022E0F57308
:1034190002211F02212102212602213A02213F0213
:10342900214402214902214E02215302215802213D
:073439005D02216202216720
:10216D009006DEE0FE9006DFE0D39E404B9006DD4C
:10217D00E0B404189006DFE0C395735002D233909B
:10218D0006DEE0D395734002C233802A9006DEE06E
:10219D00C3957350099006DFE0D39573500280020A
:1021AD00D2339006DEE0D3957350099006DFE0C37D
:1021BD0095735002C233802A9006DEE0D3957340AA
:1021CD00099006DFE0C3957340028002C23390068A
:1021DD00DEE0C3957340099006DFE0D395734002AE
:1021ED00D233229006E1E0903440F8282873804CD9
:1021FD0085537380479000E9E0855FF0A4FFAEF052
:10220D0074081200398F738033856173802E856752
:10221D007380298568738024856973801F856A732F
:10222D00801A856B73801585667380108565738044
:0C223D000B856C738006900022E0F573A6
:103440000221FB0221FD02220202221602221B029D
:10345000222002222502222A02222F0222340222C4
:073460003902223E02224363
:102249009006E2E0FE9006E3E0D39E405F9006E14F
:10225900E0B404189006E3E0C395735002D23490B9
:1022690006E2E0D395734002C234803E9006E2E074
:10227900C3957350099006E3E0D395735002800229
:10228900D2349006E2E0D3957350099006E3E0C397
:1022990095735002C2349006E1E0B401099000F54B
:1022A900E0D3956150028002C234802A9006E2E0B0
:1022B900D3957340099006E3E0C395734002800209
:1022C900C2349006E2E0C3957340099006E3E0D377
:1022D90095734002D234229006E5E0903467F828DD
:1022E9002873804C85537380479000E9E0855FF03F
:1022F900A4FFAEF074081200398F738033856173BF
:10230900802E856773802985687380248569738029
:102319001F856A73801A856B7380158566738010B3
:10232900856573800B856C738006900022E0F573D8
:103467000222EB0222ED0222F202230602230B02C2
:10347700231002231502231A02231F0223240223E7
:073487002902232E0223336A
:102339009006E6E0FE9006E7E0D39E404B9006E566
:10234900E0B404189006E7E0C395735002D23590C3
:1023590006E6E0D395734002C235802A9006E6E08E
:10236900C3957350099006E7E0D395735002800234
:10237900D2359006E6E0D3957350099006E7E0C39D
:1023890095735002C235802A9006E6E0D3957340D2
:10239900099006E7E0C3957340028002C2359006B2
:1023A900E6E0C3957340099006E7E0D395734002D0
:1023B900D235229006E9E090348EF8282873804CB3
:1023C90085537380479000E9E0855FF0A4FFAEF084
:1023D90074081200398F738033856173802E856785
:1023E9007380298568738024856973801F856A7362
:1023F900801A856B73801585667380108565738077
:0C2409000B856C738006900022E0F573D8
:10348E000223C70223C90223CE0223E20223E7024C
:10349E0023EC0223F10223F60223FB022400022472
:0734AE000502240A02240FAD
:102415009006EAE0FE9006EBE0D39E404B9006E97D
:10242500E0B404189006EBE0C395735002D23690E1
:1024350006EAE0D395734002C236802A9006EAE0A8
:10244500C3957350099006EBE0D395735002800253
:10245500D2369006EAE0D3957350099006EBE0C3B7
:1024650095735002C236802A9006EAE0D3957340F0
:10247500099006EBE0C3957340028002C2369006D0
:10248500EAE0C3957340099006EBE0D395734002EB
:10249500D236229006EDE09034B5F8282873804CAA
:1024A50085537380479000E9E0855FF0A4FFAEF0A7
:1024B50074081200398F738033856173802E8567A8
:1024C5007380298568738024856973801F856A7385
:1024D500801A856B7380158566738010856573809A
:0C24E5000B856C738006900022E0F573FC
:1034B5000224A30224A50224AA0224BE0224C302D4
:1034C50024C80224CD0224D20224D70224DC0224FB
:0734D500E10224E60224EBF2
:1024F1009006EEE0FE9006EFE0D39E404B9006ED95
:10250100E0B404189006EFE0C395735002D23790FF
:1025110006EEE0D395734002C237802A9006EEE0C2
:10252100C3957350099006EFE0D395735002800272
:10253100D2379006EEE0D3957350099006EFE0C3D1
:1025410095735002C237802A9006EEE0D39573400E
:10255100099006EFE0C3957340028002C2379006EE
:10256100EEE0C3957340099006EFE0D39573400206
:10257100D237229006F1E09034DCF8282873804CA1
:1025810085537380479000E9E0855FF0A4FFAEF0CA
:1025910074081200398F738033856173802E8567CB
:1025A1007380298568738024856973801F856A73A8
:1025B100801A856B738015856673801085657380BD
:0C25C1000B856C738006900022E0F5731F
:1034DC0002257F02258102258602259A02259F025C
:1034EC0025A40225A90225AE0225B30225B8022582
:0734FC00BD0225C20225C735
:1025CD009006F2E0FE9006F3E0D39E404B9006F1AC
:1025DD00E0B404189006F3E0C395735002D238901E
:1025ED0006F2E0D395734002C238802A9006F2E0DD
:1025FD00C3957350099006F3E0D395735002800292
:10260D00D2389006F2E0D3957350099006F3E0C3EB
:10261D0095735002C238802A9006F2E0D39573402C
:10262D00099006F3E0C3957340028002C23890060C
:10263D00F2E0C3957340099006F3E0D39573400221
:10264D00D238229006F5E0903503F8282873804C97
:10265D0085537380479000E9E0855FF0A4FFAEF0ED
:10266D0074081200398F738033856173802E8567EE
:10267D007380298568738024856973801F856A73CB
:10268D00801A856B738015856673801085657380E0
:0C269D000B856C738006900022E0F57342
:1035030002265B02265D02266202267602267B02E3
:10351300268002268502268A02268F022694022608
:073523009902269E0226A377
:1026A9009006F6E0FE9006F7E0D39E404B9006F5C3
:1026B900E0B404189006F7E0C395735002D239903C
:1026C90006F6E0D395734002C239802A9006F6E0F7
:1026D900C3957350099006F7E0D3957350028002B1
:1026E900D2399006F6E0D3957350099006F7E0C306
:1026F90095735002C239802A9006F6E0D39573404B
:10270900099006F7E0C3957340028002C23990062A
:10271900F6E0C3957340099006F7E0D3957340023C
:10272900D239229006F9E090352AF8282873804C8E
:1027390085537380479000E9E0855FF0A4FFAEF010
:1027490074081200398F738033856173802E856711
:102759007380298568738024856973801F856A73EE
:10276900801A856B73801585667380108565738003
:0C2779000B856C738006900022E0F57365
:10352A0002273702273902273E022752022757026B
:10353A00275C02276102276602276B02277002278F
:07354A007502277A02277FBA
:102785009006FAE0FE9006FBE0D39E404B9006F9DA
:10279500E0B404189006FBE0C395735002D23A905A
:1027A50006FAE0D395734002C23A802A9006FAE011
:1027B500C3957350099006FBE0D3957350028002D0
:1027C500D23A9006FAE0D3957350099006FBE0C320
:1027D50095735002C23A802A9006FAE0D395734069
:1027E500099006FBE0C3957340028002C23A900649
:1027F500FAE0C3957340099006FBE0D39573400258
:10280500D23A229006FDE0903551F8282873804C85
:1028150085537380479000E9E0855FF0A4FFAEF033
:1028250074081200398F738033856173802E856734
:102835007380298568738024856973801F856A7311
:10284500801A856B73801585667380108565738026
:0C2855000B856C738006900022E0F57388
:1035510002281302281502281A02282E02283302F3
:10356100283802283D02284202284702284C022816
:073571005102285602285BFD
:102861009006FEE0FE9006FFE0D39E404B9006FDF1
:10287100E0B404189006FFE0C395735002D23B9078
:1028810006FEE0D395734002C23B802A9006FEE02B
:10289100C3957350099006FFE0D3957350028002EF
:1028A100D23B9006FEE0D3957350099006FFE0C33A
:1028B10095735002C23B802A9006FEE0D395734087
:1028C100099006FFE0C3957340028002C23B900667
:1028D100FEE0C3957340099006FFE0D39573400273
:1028E100D23B22900701E0903578F8282873804C7C
:1028F10085537380479000E9E0855FF0A4FFAEF057
:1029010074081200398F738033856173802E856757
:102911007380298568738024856973801F856A7334
:10292100801A856B73801585667380108565738049
:0C2931000B856C738006900022E0F573AB
:103578000228EF0228F10228F602290A02290F027E
:10358800291402291902291E02292302292802299D
:073598002D02293202293740
:10293D00900702E0FE900703E0D39E404B90070105
:10294D00E0B40418900703E0C395735002D23C9095
:10295D000702E0D395734002C23C802A900702E043
:10296D00C395735009900703E0D39573500280020D
:10297D00D23C900702E0D395735009900703E0C352
:10298D0095735002C23C802A900702E0D3957340A4
:10299D0009900703E0C3957340028002C23C900783
:1029AD0002E0C395734009900703E0D3957340028D
:1029BD00D23C22AE2FAF3074F5D39F74019E4008E8
:1029CD00782F126B99022ADA753001752F00AE52ED
:1029DD00AF53E547BE000DD39F40099000CBE0D328
:1029ED00954840028023754800E547C39553F5731C
:1029FD009000CEE0D395464008E5462573F5468018
:102A0D00069000CEE0F546800205489000A7E0D381
:102A1D009561401CE55FC395604015AE52AF53E51F
:102A2D0047BE00039F50099000CCE0D3954940026A
:102A3D00806E9007E3E0A852B800049553500375DB
:102A4D004B009007E3E0A852B8000BD39553400616
:102A5D00E5539007E3F0E54B7041E553C39547F51A
:102A6D0073E573D3940540037573059000CDE0C3F2
:102A7D0095465007E573C3954640028009E546C368
:102A8D009573F54680069000CDE0F5469000CDE0BB
:102A9D00D3954640069000CDE0F54675490080027D
:102AAD000549E54B70169000A7E0C39561500DE503
:102ABD00472405A852B8000695534002800F900098
:102ACD00BAE0F546754B0174789007E3F022AE2F0E
:102ADD00AF3074E9D39F74039E4008782F126B9921
:102AED00022C79753001752F00754632A23D402AB2
:102AFD007546199000BAE075F002A4FFAEF0E548F6
:102B0D00BE0006D39F4002D23D0548754B03747835
:102B1D009007E3F0754A00022C68AE52AF53E547BB
:102B2D006F4E7003022C68E547BE000DD39F400920
:102B3D009000CBE0D395484002800F754800E54BDF
:102B4D00C394035003754619800DE547C39553F59E
:102B5D0073E5482573F5489000A7E0D39561400EC5
:102B6D009007E3E0A852B80007D395534002800CBC
:102B7D00054A9000BAE0B54A03754B00E54BB40326
:102B8D0006A20BB3B34002800A054AE54AB43C03E2
:102B9D00754B02E54BB402299007E3E0A852B8004B
:102BAD000ED395534009E5539007E3F0754A009015
:102BBD0000A7E0C395615009754A0074789007E34A
:102BCD00F0E54B705A9000A7E0D39561401CE55F8E
:102BDD00C395604015AE52AF53E547BE00039F50FD
:102BED00099000CCE0D395494002800875490075E5
:102BFD00464B8028E553C39547F573E573D394058C
:102C0D0040037573059000A7E0D395614008E54931
:102C1D002573F5498006E5492406F549754A00E511
:102C2D004B70169000A7E0C39561500DE547240544
:102C3D00A852B80006955340028003754B01E54B31
:102C4D00B40118754619054A9000BAE0B54A0675E3
:102C5D004B02754A0074789007E3F0E54675F00A6B
:102C6D00A4FFAEF09007D8EEF0A3EFF022E56F9041
:102C7D00359FF828287390009FE07003022E28904E
:102C8D0000D5E0B401028003022D78900063E0B519
:102C9D005E028003022D757E017F00E5BE126B453D
:102CAD00E5BD2FFF50010E8E5A8F5B7410126B45D0
:102CBD0090008EE08E048F05FF126B359007E4ECCB
:102CCD00F0A3EDF0E56B60089000FBE0640260029C
:102CDD0080269000FDE0B4011F9007E4E0FEA3E024
:102CED00FF74E7126B45E56B8E048F05FF126B3594
:102CFD009007E4ECF0A3EDF090009FE0B402279074
:102D0D0007E6E0FEA3E0FF9007E4E0FCA3E0FDEFA3
:102D1D002DFDEE3CFC74018C068D071200399007D9
:102D2D00E4EEF0A3EFF09007E4E0FEA3E0FF9007E0
:102D3D00E6E0FCA3E0FDEDD39FEC9E4004D2408085
:102D4D0002B2409007E4E0F8A3E09007E6C8F0A3D4
:102D5D00C8F09000D1E064016006A240B3B3400218
:102D6D0080069007E5E0F55F022E26D2407E017FBA
:102D7D0000E5BE126B45E5BD2FFF50010E8E5A8F3B
:102D8D005B7410126B4590008EE08E048F05FF1260
:102D9D006B359007E4ECF0A3EDF0E56B6008900067
:102DAD00FBE06402600280269000FDE0B4011F90FC
:102DBD0007E4E0FEA3E0FF74E7126B45E56B8E04BC
:102DCD008F05FF126B359007E4ECF0A3EDF090004A
:102DDD009FE0B402279007E6E0FEA3E0FF9007E432
:102DED00E0FCA3E0FDEF2DFDEE3CFC74018C068DA7
:102DFD00071200399007E4EEF0A3EFF09007E4E03E
:102E0D00F8A3E09007E6C8F0A3C8F09000D1E06405
:102E1D000160069007E5E0F55F8003755F009000A7
:102E2D009BE07006756F01022C7A75BB180233F3A7
:102E3D0090009BE07003022FC97E017F00E5BE125A
:102E4D006B45E5BD2FFF50010E8E5A8F5B9000E153
:102E5D00E0B4010F7E0F7FFFAC5AAD5B126B918E0C
:102E6D005A8F5B900106E0B40245AE5AAF5B9000FD
:102E7D002BE0FCA3E0FDEDD39FEC9E400A90002BD0
:102E8D00E55AF0A3E55BF0AE5AAF5B90002DE0FC88
:102E9D00A3E0FDEFD39DEE9C400A90002DE55AF086
:102EAD00A3E55BF0AE5AAF5B74041200398F6190ED
:102EBD000106E0704CAE5AAF5B90002BE0FCA3E036
:102ECD00FDEFD39DEE9C4009126B918E5A8F5B8066
:102EDD0006755B00755A00AE5AAF5B7410126B45E8
:102EED0090008BE08E048F05FF126B358C5A8D5B35
:102EFD0074FFBC0009D39D4005855B61800375613E
:102F0D00FE9000D1E0B401028003022FC7A20BB3E3
:102F1D00B3500E9000A5E0A852B80005D3955350BC
:102F2D0003022FBC9000A6E075F019A4FFAEF0903F
:102F3D0000E9E08E048F05FF126B359000E2E0850D
:102F4D0061F0A4FFAEF074648D028C038E048F05C6
:102F5D00FF126B35EA2DFDEB3CFC8C5A8D5BE56B5E
:102F6D00600F9000FBE0B402089000FDE06401608A
:102F7D00028017AE5AAF5B74E7126B45E56B8E049A
:102F8D008F05FF126B358C5A8D5BAE5AAF5B900778
:102F9D00E4E0FCA3E0FDEDD39FEC9E4005855B5F77
:102FAD00800BA240B340069007E5E0F55F800BA2D1
:102FBD0040B340069007E5E0F55F80037561009032
:102FCD00009EE07006756F02022C7A75BB190233F4
:102FDD00F390009EE0700302307EE55ED395514084
:102FED000302307C900029E0FEA3E0FFE565126B43
:102FFD0089900029EEF0A3EFF07E017F00E5BE126F
:10300D006B45E5BD2FFF50010E8E5A8F5B90010B66
:10301D00E07013740A126B4574518E048F05FF1204
:10302D006B358D658019AE5AAF5B740A126B458F87
:10303D00048E057E017F95CDCCCD126A338F65E56B
:10304D0065D394644003756564900029E0FEA3E0A8
:10305D00FFE5652FFF50010E900029EEF0A3EFF074
:10306D009000A2E0048E048F05FF126B358D6580F4
:10307D00037565329000EEE07006756F03022C7AD1
:10308D0075BB130233F39000EEE0604A7E017F00C2
:10309D00E5BE126B45E5BD2FFF50010E8E5A8F5BBD
:1030AD0074041200398F669000F0E08566F0A4FD7F
:1030BD00ACF07464FF126B358D669000EFE08566A1
:1030CD00F0A4FFAEF074FF8E048F05FF126B35ED8B
:1030DD0090008AF0800375660090009CE070067584
:1030ED006F04022C7A75BB170233F390009CE0B489
:1030FD000102800302318C7E017F00E5BE126B451B
:10310D00E5BD2FFF50010E8E5A8F5B9007E8E060F2
:10311D00199007E8E0149064B112008CE493FC74EC
:10312D000193FDEDC39FEC9E400280069007E8E001
:10313D0014F09007E8E0C394B3501DAE5AAF5B9006
:10314D0007E8E0049064B112008CE493FC740193E1
:10315D00FDEFC39DEE9C400280069007E8E004F071
:10316D009007E8E0FE9000C2E08E0088F0A4FFAE6C
:10317D00F074648E048F05FF126B358D67800375B7
:10318D00670090009DE07006756F05022C7A75BB87
:10319D00160233F390009DE0B40102800302323534
:1031AD007E017F00E5BE126B45E5BD2FFF50010E80
:1031BD008E5A8F5B9007E9E060199007E9E0149053
:1031CD00661B12008CE493FC740193FDEDC39FEC20
:1031DD009E400280069007E9E014F09007E9E0C3F5
:1031ED0094B3501DAE5AAF5B9007E9E00490661B97
:1031FD0012008CE493FC740193FDEFC39DEE9C4093
:10320D000280069007E9E004F09007E9E0FE9000E7
:10321D00C8E08E0088F0A4FFAEF074648E048F05B4
:10322D00FF126B358D68800375680075BB1F023307
:10323D00F37E017F00E5BE126B45E5BD2FFF50010A
:10324D000E8E5A8F5B7409126B4574E68E048F05D2
:10325D00FF126B358D6A9000A4E07006756F070242
:10326D002C7A75BB150233F39000A4E07003023382
:10327D008F7E017F00E5BE126B45E5BD2FFF50012E
:10328D000E8E5A8F5B74041200398F699000A4E082
:10329D00B401159000F8E08569F0A4FFAEF0740755
:1032AD00120039EF9007DDF09000A4E0B402159004
:1032BD0000F8E08569F0A4FFAEF07407120039EF55
:1032CD009007DCF09000A4E0B40302800302338D7C
:1032DD009000E5E070389000F8E0601CE569C3945B
:1032ED00195002D232E569D394644002C232900083
:1032FD00C4E09007E0F08014E569C394195002D240
:10330D0041E569D394324002C241C23280639000DC
:10331D00C4E070349000F8E08569F0A4FFAEF0745D
:10332D00FF8E048F05FF126B35ED9007E0F0AE5266
:10333D00AF53741EBE0006D39F4002D232E561D357
:10334D0094E54002C2328029E569C3940A500DAE5E
:10335D0052AF53741EBE0004D39F50028002D2326E
:10336D00E561D394E54002C2329000C4E09007E0DD
:10337D00F09007E0E0C39405500674059007E0F067
:10338D0080037569009000FBE07006756F08022CD4
:10339D007A75BB1480509000FBE060397E017F0090
:1033AD00E5BE126B45E5BD2FFF50010E8E5A8F5BAA
:1033BD00EFD39421EE940E4005756BFF8015AE5A38
:1033CD00AF5B7410126B4574E38E048F05FF126BA7
:1033DD00358D6B8003756B0090009FE0600575BBAC
:0633ED001A800375BB18F5
:10359F00022C83022E3D022FDE0230930230F802FE
:0B35AF0031A102323E0232750233A34C
:0533F300056FD2EC2281
:096B77002582F5825002058322FB
:0F008C0025E050020583258250020583F582226C
:106B1400EF2F500205832582F582E5833E2EF5830F
:016B2400224E
:106B8900CFC39FFF50011E22C3EF9DFFEE9CFE2243
:086B99000806B60002180622EE
:0D6B5300A3E004F07006120049E004F022F7
:0E003900048007C3CE13CECF13CFD5E0F6223E
:106A3300BC000FBE0008ED8FF084FFADF022E4FE32
:106A4300FF22BE000DEF60FE54F0606F20E70302EB
:106A53006AE9EAC0E0EBC0E078017A0075F001EE84
:106A630020E710EF25E0FFEE33FE0AC5F023C5F063
:106A730030E7F0EA5407F9096A7A007B00600108FD
:106A8300C3EC9E40167004ED9F4010ED9FFDEC9EFD
:106A9300FCE5F0CA4ACA03F5F08005E5F003F5F01A
:106AA300C3EE13FEEF13FFD9D77908CACBCAD8D0E8
:106AB300EAFEEBFFD0E0FBD0E0FA22EC8FF084FC9F
:106AC300ED54F045F0C48FF084FEEDC454F045F06E
:106AD300C48FF084FDEEC4FE54F02DFFEE540F3C42
:106AE300FEADF07C0022790078008FF0EC7E082068
:106AF300E70DC3CD33CD33C933C9C833C8DEF08402
:106B030049F9E5F08FF0BE00E6FD7C00E9FFE8FE01
:016B1300225F
:0E6B4500F88FF0A4FFE5F0CE88F0A42EFE221B
:10000300EF8DF0A4F9A8F0EF8CF0A428F8EE8DF0B2
:06001300A428FEE9FF2213
:106B2500600D782B026B2F007830D8FED5E0F82267
:106B3500EEC0E07E00126A33EFFDEEFCD0E0FE22EF
:0C6B6000EEC0E07E00126A33D0E0FE229E
:03001B0002001EC2
:0300530002005652
:03009B00020071EF
:03000000026B8010
:096B800075817575D00002409D7D
:0B6B6C00E5822FF582E5833EF58322D1
:0A0049000582D5820215831582227C
:10001E00C0E0C0F0C083C082C0D075D00012404A8C
:0B002E00D0D0D082D083D0F0D0E032E0
:10005600C0E0C0F0C083C082C0D075D00012404D51
:10006600D0D0D082D083D0F0D0E032C0E0C0F0C093
:1000760083C082C0D075D00012406DD0D0D082D05F
:0600860083D0F0D0E0324F
:00000001FF
